:0408000074EF50F051
:08080800046ED8CF05F0E0CF2B
:1008100006F00001E9CF0CF0EACF07F0E1CF08F0D5
:10082000E2CF09F0D9CF0AF0DACF0BF0F3CF12F014
:10083000F4CF13F0FACF14F0F5CF15F0F6CF16F091
:10084000F7CF17F000C00EF001C00FF002C010F09B
:1008500003C011F0F2AA30EF04F0F2B417EF1FF06A
:100860000EC000F00FC001F010C002F011C003F084
:100870000CC0E9FF07C0EAFF078E08C0E1FF09C00E
:10088000E2FF0AC0D9FF0BC0DAFF12C0F3FF13C0AA
:10089000F4FF14C0FAFF15C0F5FF16C0F6FF17C02D
:1008A000F7FF045006C0E0FF05C0D8FF1000254345
:1008B000315D2050726F6772616D20426C61636BB5
:1008C00020202020202020325D2050726F6772612E
:1008D0006D204379616E2020202020202020335D70
:1008E0002050726F6772616D204D6167656E746133
:1008F000202020202025430D0A002543345D205070
:10090000726F6772616D2059656C6C6F7720202063
:10091000202020355D2050726F6772616D204C2F52
:100920004379616E202020202020365D2050726F98
:100930006772616D204C2F4D6167656E7461202078
:100940002025430D0A002543375D2050726F6772E2
:10095000616D2057686974652020202020202020A8
:100960002020202020202020202020202020202087
:100970002020202020202020202020202020202077
:100980002020202020202020202020202025430D52
:100990000A0025432D2D2D2D2D2D2D2D2D2D2D2DC9
:1009A0002D2D2D2D2D2D2D2D2D2D2D2D2D2D2D2D77
:1009B0002D2D2D2D2D2D2D2D2D2D2D2D2D2D2D2D67
:1009C0002D2D2D2D2D2D2D2D2D2D2D2D2D2D2D2D57
:1009D0002D2D2D2D2D2D2D2D2D25430D0A0025439B
:1009E000415D20526561642055494420202020202B
:1009F00020202020202020425D2053656172636802
:100A00002055494420202020202020202020435D04
:100A100020526561642064617461206D656D6F7240
:100A2000792020202025430D0A002543445D2057CE
:100A3000726974652074686520535020202020203E
:100A4000202020455D205265616420746865205334
:100A50002F506164202020202020465D2053686FA5
:100A6000772063726564697473207374617475733D
:100A70002025430D0A002543475D205265636861C8
:100A80007267652043726564697473202020204872
:100A90005D20436F707920535020746F204D656D39
:100AA0006F7279202020495D205265616420417079
:100AB0006C2E207265676973746572202025430D62
:100AC0000A0025434A5D2057726974652041706CA5
:100AD0002E207265676973746572204B5D20436FC9
:100AE00070792041706C2E2072656769737465722D
:100AF00020204C5D20436F70792041706C2E207255
:100B000065676973746572202025430D0A002543CB
:100B10004D5D205265616420537461747573206269
:100B2000797465202020204E5D2052657365742DF8
:100B300041434B20546573742020202020204F5DBA
:100B4000204368616E67652053657373696F6E201B
:100B5000202020202025430D0A002543505D2043FE
:100B60006F70792044657669636520496D616765BA
:100B7000202020515D2050617374652044657669A2
:100B8000636520496D6167652020525D20546F6761
:100B900067656C20546172676574206368697020B2
:100BA0002025430D0A002543535D2050676D2E20FC
:100BB0004578706972652064617465202020205436
:100BC0005D20526561642062756C6B20696E6B20DC
:100BD0006C6576656C20595D204D656D6F7279206E
:100BE00064756D7028524157292020202025430D1F
:100BF0000A002543555D20536574205549442073F0
:100C00007461727420706F696E7420565D20536534
:100C100074206D66672E206461746520202020207A
:100C20002020585D20456E67696E656572696E6744
:100C3000206F7074696F6E732025430D0A00254381
:100C4000415D2052656164207468652055494420E7
:100C500020202020202020435D20526561642064F4
:100C6000617461206D656D6F727920202020455D73
:100C700020526561642074686520532F50616420A0
:100C8000202020202025430D0A002543465D2053C7
:100C9000686F77204372656469747320737461743C
:100CA000757320475D2052656368617267652043F4
:100CB00072656469747320202020495D205265614B
:100CC000642041706C2E20726567697374657220B0
:100CD0002025430D0A0025434D5D205265616420A7
:100CE0005374617475732062797465202020204FDD
:100CF0005D204368616E67652053657373696F6E2D
:100D0000202020202020505D20436F7079204465F2
:100D10007669636520496D61676520202025430D54
:100D20000A002543515D2050617374652044657647
:100D300069636520496D6167652020565D205365B4
:100D400074206D66672E2064617465202020202049
:100D50002020535D2050676D2E20457870697265A4
:100D600020646174652020202025430D0A0025435E
:100D7000525D20546F6767656C20546172676574BB
:100D800020636869702020575D2053796E6320636B
:100D900068697020746F20696E6B20202020585D78
:100DA00020456E67696E656572696E67206F707445
:100DB000696F6E732025430D0A000D0A2020202044
:100DC0003030203031203032203033203034203069
:100DD000352030362030372030382030392030412F
:100DE0002030422030432030442030452030460D12
:100DF0000A004379616E202020202020202020201E
:100E000020004D6167656E74612020202020202025
:100E1000200059656C6C6F77202020202020202036
:100E20002000426C61636B202020202020202020A5
:100E300020004C69676874204379616E202020206F
:100E400020004C69676874204D6167656E7461208D
:100E50002000576869746520202020202020202051
:100E60002000556E646566696E656420636F6C6F03
:100E70007200526F6C616E642000302E2E4D696DD1
:100E8000616B69204A563328535331292020202092
:100E900020312E2E4D696D616B69204A56332853DF
:100EA000533229202020202020322E2E4D696D61C2
:100EB0006B69204A563528485329202020200D0AE6
:100EC0000000332E2E4A5633332853533231292013
:100ED000202020202020202020342E2E4A5633335C
:100EE0002842532D3229202020202020202020207D
:100EF00020352E2E4A56352F33332853423531298B
:100F00002020202020200D0A0000362E2E4A5635A3
:100F10002F3333285342353229202020202020200F
:100F200020372E2E4A5633332845532D332920207F
:100F3000202020202020202020382E2E554A4628F0
:100F40004C46313030293232306D6C2020200D0A71
:100F50000000392E2E554A46284C4831303029366B
:100F600030306D6C2020202020412E2E554A562FE7
:100F70004A4658284C46323030293630306D6C2085
:100F800020422E2E554A46284C46323030293232E5
:100F9000306D6C2020200D0A0000432E2E4A462F73
:100FA0004A46532855562920202020202020202042
:100FB0002020202020202020202020202020202031
:100FC0002020202020202020202020202020202021
:100FD00020202020202020202020202020200D0A3A
:100FE000000046757475726520546563686E6F6C99
:100FF0006F6769657300536F757468204166726925
:10100000636100002B2B32373231203937362D35D2
:1010100038313100202020202020202020202020B6
:101020007777772E467574757265746563686E6F31
:101030006C6F676965732E636F2E7A6100000D45D2
:1010400052524F523A2054686520312D57697265CB
:101050002062757320686173206E6F20766F6C74E8
:1010600061676520737570706C7900000D45525290
:101070004F523A20546865205245534554207075AC
:101080006C7365206973206E6F74206265696E678A
:101090002041434B6E6F776C6564676564000D5249
:1010A00065747279696E672E2E2020202020202002
:1010B0002020202020202020202020202020202030
:1010C0002020202020202020202020202020200040
:1010D00046616D696C7920436F64653A202532580A
:1010E000202049443A200000204352433A20253230
:1010F000580D0A000D0A204E6F20646576696365FD
:1011000073206F6E2074686520312D5769726520D9
:10111000627573002532553A2D2020002532553A4C
:101120002D2020000D0A4465766963652F732070B9
:10113000726573656E742C20627574206E6F7420F6
:10114000746865206D756C74692D64726F7020769B
:1011500061726965747900000D0A456E74657220CC
:101160007768696368206465766963652773206DB5
:10117000656D6F727920697320746F2062652069D4
:101180006E746572726F67617465642E2042792097
:10119000656E746572696E672061206E756D62653B
:1011A00072206E6F74000D0A6C6973746564207729
:1011B000696C6C2070726576656E74206120737046
:1011C00065636966696320646576696365206F6E2F
:1011D00020746865206D756C746964726F7020622C
:1011E00075732066726F6D206265696E67000D0A07
:1011F0006163746976617465642E20000D455252F6
:101200004F523A2054686520312D5769726520622B
:10121000757320686173206E6F20766F6C746167E0
:101220006520737570706C7900000D0A0A52657341
:1012300065743A25752041434B27733A25750D0A8D
:1012400000000D4552524F523A2054686520312D0E
:10125000576972652062757320686173206E6F2014
:10126000766F6C7461676520737570706C790000BF
:101270000D0A0A52657365743A25752041434B2760
:10128000733A25750D0A00000D0A507265737320BC
:10129000616E79206B657920746F20636F6E74695D
:1012A0006E75652E2E2E0000202020202563000064
:1012B000202020202563204D61696E204D656E75CC
:1012C000202D20004D696D616B69204A462F4A46EA
:1012D0005328555629202020202000004D696D619B
:1012E0006B69204A5633285353312920202020206F
:1012F000202000004D696D616B69204A56332853E8
:101300005332292020202020202000004D696D61CB
:101310006B69204A5633332845532D335F202020F4
:10132000202000004D696D616B69204A56352848C0
:101330005329202020202020202000004D696D61AD
:101340006B69204A56352F333328534235312F35B8
:10135000322900004D696D616B69204A563333288C
:101360005353323129202020202000004D696D6127
:101370006B69204A5633332842532D3229202020CE
:10138000202000004D696D616B69204C483230307F
:101390002073657269657320202000004D696D61BE
:1013A0006B69204C4631303020736572696573205B
:1013B00020200000526F6C616E642045636F736F74
:1013C0006C7665202020202020200000556E64656A
:1013D00066696E6564204F454D2020202020202026
:1013E000202000004E6F206368697020646574657A
:1013F00063746564202020202020202020202020CD
:1014000020202020202020202020200020202020FC
:101410002020202025630000202A2A2A2A204D6926
:101420006D616B69204A56332D5479706520496E81
:101430006B204361727472696467652052657365DD
:101440007474696E672F50726F6772616D6D696E2B
:1014500067204465766963652052657620312E34B5
:1014600035202A2A2A2A0D0A0000202020202020A8
:10147000202020200000202D2054656C3A002020E0
:101480002020202020202020202020200000204379
:10149000757272656E742053657373696F6E3A204E
:1014A00000004D696D616B6920004A563328535323
:1014B000312900004A5633285353322900004A5636
:1014C0003528485329004A5633332853533231299B
:1014D00000004A5633332842532D322900004A5621
:1014E000352F33332853422D353129004A56352FB5
:1014F00033332853422D35322900554A46284C466D
:10150000313030290000554A46284C4831303029C6
:101510000000554A562F4A4658284C46323030294A
:101520000000554A46284C463230302900004A46D1
:101530002F4A4653285556290000456E646C657342
:10154000730020202044617465207365743A200084
:101550002020205461726765743A20000D0A53659B
:101560006C656374206F7074696F6E3A20200000A0
:101570004465766963652053657269616C204E75B8
:101580006D6265723A256C75202D20526573657405
:10159000206C6F673A25750D0A0A000028506C65AB
:1015A000617365204E4F54453A207468652061622E
:1015B0006F766520696E666F726D6174696F6E20FB
:1015C0006D7573742062652071756F746564207722
:1015D00068656E2070757263686173696E672063F9
:1015E0007265646974732E0D0A005468697320690A
:1015F0006E666F726D6174696F6E206973207573AA
:10160000656420746F2067656E6572617465206122
:10161000206B657920746861742077696C6C206236
:10162000652073656E74206261636B20746F20792E
:101630006F752E290D0A0A00437265646974732060
:1016400072656D61696E696E673A20256C750D0A69
:101650000A000D0A456E74657220746865206E7507
:101660006D626572206F66207265736574206372A7
:101670006564697473206265696E67207075726352
:1016800068617365643A2D2020000D0A456E74650B
:1016900072207468652034302063686172616374FD
:1016A0006572206B6579636F646520737570706C0B
:1016B00069656420627920003A2D200D0A000D0A28
:1016C0005265736574206372656469747320616D1B
:1016D0006D656E64656420737563636573736675A9
:1016E0006C6C792066726F6D20256C7520746F208C
:1016F000256C752E00000D0A496E76616C696420B8
:10170000636F64652E002A2A2A2A00005220452091
:101710005320452054005720522049205420452072
:10172000202020502052204F20432045205320537A
:1017300000002020205320552043204320452053E3
:1017400020462055204C2A2A2A2A00000A0A0D5237
:101750004553455420636F756E746572206973201C
:1017600061646A757374656420746F3A20256C75C2
:101770000A0D00000D0A20284E6F2063726564690F
:1017800074732072656D61696E696E672E20507585
:10179000726368617365206372656469747320663F
:1017A000726F6D2046542E290D0A00004341555496
:1017B000494F4E2120596F75206F6E6C79206861FA
:1017C000766520256C7520637265646974002072EB
:1017D000656D61696E696E672E2050757263686110
:1017E000736520637265646974732066726F6D201F
:1017F0000D0A0000206265666F726520796F757250
:10180000206372656469747320636F756E746572AA
:101810002072656163686573207A65726F2E0000BF
:1018200020202020202044533234333041203235D0
:10183000362D426974204D656D6F72790D0A000076
:101840002020202020202D2D2D2D2D2D2D2D2D2D16
:101850002D2D2D2D2D2D2D2D2D2D2D2D0D0A000055
:101860000D0A0A20202020496E6B204C6576656C9D
:101870003A002020204578706972652064617465A3
:101880003A200000202D20436865636B73756D203E
:101890004572726F7220253258202532580020433D
:1018A0006F7272656374656421000D0A496E70750C
:1018B0007420746865207374617274696E67206146
:1018C0006464726573733A2D20000D0A4E756D6263
:1018D0006572206F6620627974657320746F20775B
:1018E000726974653A2D20000D0A496E7075742076
:1018F00064617461206279746520666F722061642E
:101900006472657373202532583A2D2000000D0A49
:1019100053637261746368706164206973207472C8
:10192000616E7366657272656420746F206D656D9B
:101930006F72792E2E000D0A5374617475732044F2
:101940006174613A2D2030782532582000000D0A4C
:10195000284170706C69636174696F6E20526567AD
:101960006973746572206973206C6F636B65642999
:1019700000000D0A284170706C69636174696F6EB4
:101980002052656769737465722069732073746986
:101990006C6C20756E6F636B656429000D0A2020E6
:1019A000202030302030312030322030332030348D
:1019B000203035203036203037000D0A20202020FE
:1019C00000000D0A436F7069656420616E64206CCD
:1019D0006F636B656420746865206170706C696307
:1019E0006174696F6E2072656769737465722E0A1F
:1019F000000020202020202050726F6772616D202F
:101A0000746865204170706C69636174696F6E20E1
:101A100052656769737465720D0A000020202020EA
:101A200020202D2D2D2D2D2D2D2D2D2D2D2D2D2D00
:101A30002D2D2D2D2D2D2D2D2D2D2D2D2D2D2D2DD6
:101A40002D2D0D0A00000D0A496E70757420746802
:101A500065207374617274696E6720616464726575
:101A600073733A2D20000D0A4E756D626572206FFA
:101A70006620627974657320746F2077726974656B
:101A80003A2D20000D0A496E7075742064617461EE
:101A9000206279746520666F722061646472657378
:101AA00073202532583A2D2000000D0A496E7365C7
:101AB00072742061206368697020616E64207072A6
:101AC00065737320616E79206B657920746F206374
:101AD0006F6E74696E75652E2E2E00000D0A4E6FA6
:101AE0007720636F7079696E67206368697020641E
:101AF00061746120746F20696D61676520000D0A53
:101B0000436F6D706C657465640D0A000D0A416465
:101B100064726573732070726F6772616D6D656456
:101B20003A2000002020202020205365742063618B
:101B300072747269646765204D616E756661637465
:101B400075726520446174650D0A00002020202014
:101B500020202D2D2D2D2D2D2D2D2D2D2D2D2D2DCF
:101B60002D2D2D2D2D2D2D2D2D2D2D2D2D2D2D2DA5
:101B70000D0A0000456E7465722079656172206FF0
:101B800066206D616E75666163747572652859595A
:101B90005959293A202000000D0A456E74657220BB
:101BA0006D6F6E7468206F66206D616E756661631F
:101BB000747572652831207468727520313229205D
:101BC0003A2000000D0A54686520657870697265D6
:101BD00079206461746520686173206265656E2098
:101BE0007375636365737366756C6C792063686184
:101BF0006E6765642E2E2E000D0A0A0A496E7375F3
:101C00006666696369656E7420637265646974737E
:101C100020617661696C61626C652E204368697031
:101C20002070726F6772616D6D696E672061626F9F
:101C3000727465642E2E2E000D0A41646472657301
:101C4000732070726F6772616D6D65643A20000079
:101C500020202020202053657420726573657474E1
:101C600065722070726F6772616D6D696E67205367
:101C7000657373696F6E0D0A0000202020202020FC
:101C80002D2D2D2D2D2D2D2D2D2D2D2D2D2D2D2D84
:101C90002D2D2D2D2D2D2D2D2D2D2D2D2D2D2D2D74
:101CA0000D0A00000D0A0A53656C656374207365A4
:101CB0007373696F6E3A2000204D696D616B692006
:101CC00000004A5633285353312900004A5633281E
:101CD0005353322900004A563528485329004A56A2
:101CE000333328535332312900004A5633332842C4
:101CF000532D3229000053423531284D4249532992
:101D0000000053423532284D4249532900004A56BB
:101D100033332845532D33290000554A46284C4873
:101D2000313030293232306D6C00554A46284C48EB
:101D3000313030293630306D6C00554A562F4A46C6
:101D400058284C46323030293630306D6C00554AB8
:101D500046284C46323030293232306D6C004A46CB
:101D60002F4A46532855562900004A5633285353C4
:101D7000322900000D0A0A456E7465722074686588
:101D80002063617274726964676520636170616366
:101D900069747920696E206D696C6C692D6C697449
:101DA00065727320746F2062652070726F67726154
:101DB0006D6D656420696E746F2063686970732E41
:101DC0000D0A0000284A757374203C456E746572D4
:101DD0003E20746F207573652074686520646566A5
:101DE00061756C7420636170616369747929200086
:101DF0000D0A0A0A0A0A0A0A0A000D0A596F752012
:101E0000686176652063686F73656E20746F2070FB
:101E1000726F6772616D20656E646C6573732063A9
:101E20006869707320776869636820726571756985
:101E300072652061206D696E696D756D206F662019
:101E40003330206372656469747300000D0A706535
:101E50007220636869702E20456E737572652079F3
:101E60006F7520686176652073756666696369655C
:101E70006E74206372656469747320746F20676583
:101E80006E657261746520656E646C657373206342
:101E9000686970732E002020202020205365742054
:101EA00072657365747465722053657269616C2024
:101EB0004E756D6265720D0A0000202020202020E2
:101EC0002D2D2D2D2D2D2D2D2D2D2D2D2D2D2D2D42
:101ED0002D2D2D2D2D2D2D2D2D2D0D0A000054686D
:101EE000652063757272656E7420726573657474B3
:101EF0006572205549442069732073657420746F9E
:101F00002000204845580D0A0A00456E746572206D
:101F10006120646966666572656E742076616C75B1
:101F200065206F72206A75737420707265737320F8
:101F30003C454E5445523E20746F206C6561766579
:101F40002061732069733A20000020202020202087
:101F500044657465726D696E652063686970206997
:101F60006E6B2074616E6B206C6576656C0D0A007B
:101F70002020202020202D2D2D2D2D2D2D2D2D2DDF
:101F80002D2D2D2D2D2D2D2D2D2D2D2D2D2D2D2D81
:101F90002D2D2D0D0A0A0000436172747269646769
:101FA0006520696E6B2074616E6B206C6576656C64
:101FB0002020200025354C756D6C0D0A00004275FF
:101FC0006C6B696E6B2074616E6B206C6576656CF2
:101FD0002020202020202020000025364C756D6C0C
:101FE0000D0A0A00546F74616C20696E6B2020200A
:101FF0002020202020202020202020202020000021
:1020000025364C756D6C0D0A0A00202020202020FA
:1020100053796E63726F6E697A65207468652063A8
:1020200068697020696E6B206C6576656C207769D5
:102030007468207468652061637475616C20696ED2
:102040006B207765696768740D0D0A0020202020D9
:1020500020202D2D2D2D2D2D2D2D2D2D2D2D2D2DCA
:102060002D2D2D2D2D2D2D2D2D2D2D2D2D2D2D2DA0
:102070002D2D2D2D2D2D2D2D2D2D2D2D2D2D2D2D90
:102080002D2D2D2D2D2D2D2D2D2D0D0A0A005765B1
:10209000696768207468656E20696E707574207455
:1020A00068652063757272656E742077656967680C
:1020B00074206F662061203434306D6C20696E208E
:1020C0006772616D733A200043757272656E742099
:1020D0006368697020696E6B206C6576656C3A2068
:1020E00020254C756D6C0D0A0000436F6D70757482
:1020F0006564206368697020696E6B206C65766525
:102100006C3A20254C756D6C0D0A000044696666BA
:102110006572656E63652061646A7573746D656E62
:102120007420203A20254C646D6C0D0A00000D0AC5
:102130004368697020262061637475616C20696E44
:102140006B206C6576656C20686173206265656ED6
:10215000207375636365737366756C6C792073792E
:102160006E63656420627920254C646D6C0D0A00F5
:102170000D0A4E6F206368697020262061637475B4
:10218000616C20696E6B206C6576656C206861738C
:1021900020776173206E65636365736172792E0DBC
:1021A0000A00030E0101395F0BE3010EEA6E390EDE
:1021B000E96EEF5005E002D000000400EF2EFCD7DE
:1021C0000001000C93908A900400030E0101336F0C
:1021D000F20E396F0001E5DF0101332FF9D793804B
:1021E0000400070E006E002EFED700D0938081B051
:1021F00003D0000E016E19D004006B0E006E002E8D
:10220000FED700D09380329181A032810400EF0E7E
:10221000396F0001C6DF010132A104D0010E016E49
:1022200004D003D0000E016E00D000011AEF1FF0A1
:102230001B0E04009EA8FDD7AD6E5B0E04009EA889
:10224000FDD7AD6E320E04009EA8FDD7AD6E4A0ECE
:1022500004009EA8FDD7AD6E000C01013B51016A40
:102260003A5D03E23AC100F00CD0006A080E3C6F00
:102270003A3700363B51005CD8B0006E01363C2F37
:10228000F7D70001000C015038C13AF1640E01018A
:102290003B6F0001E2DF00C038F10150300E08E171
:1022A000010139A30FD039B70DD039B9200E04D0B0
:1022B00001013997399939810126015004009EA8FE
:1022C000FDD7AD6E38C13AF10A0E3B6F0001C5DF94
:1022D00000C038F10150300E08E1010139B70CD0CF
:1022E00039A10AD039B9200E00010126015004009D
:1022F0009EA8FDD7AD6E0101300E3827385104007D
:102300009EA8FDD7AD6E0001000C1B0E04009EA818
:10231000FDD7AD6E5B0E04009EA8FDD7AD6E35C136
:1023200038F11B0E0101396F0001ADDF3B0E0400D7
:102330009EA8FDD7AD6E36C138F11B0E0101396F75
:102340000001A1DF3B0E04009EA8FDD7AD6E37C192
:1023500038F11B0E0101396F000195DF6D0E04008D
:102360009EA8FDD7AD6E000C0900F5520EE0F6CF29
:1023700038F1F7CF39F1F55004009EA8FDD7AD6EC6
:1023800038C1F6FF39C1F7FFEFD7000C1B0E040070
:102390009EA8FDD7AD6E5B0E04009EA8FDD7AD6E66
:1023A0000101386B1B0E396F00016DDF3B0E04001D
:1023B0009EA8FDD7AD6E3B0E04009EA8FDD7AD6E66
:1023C0006D0E04009EA8FDD7AD6E000CD8B204D0EF
:1023D000010EEA6E4A0EE96E006A016A026A036A39
:1023E00001014A6B4B6B4C6B4D6B495148114711C6
:1023F00046112CE0200E4E6FD890423743374437B9
:1024000045374A374B374C374D3749514D5D08E119
:1024100048514C5D05E147514B5D02E146514A5D33
:102420000FE346514A5F4751D8A0473D4B5F4851A3
:10243000D8A0483D4C5F4951D8A0493D4D5FD88058
:1024400000360136023603364E2FD6D74AC1EFFF8B
:102450004BC1ECFF4CC1ECFF4DC1ECFF0001000C87
:10246000E95001013A6F3B0E416F9A0E406FCA0E60
:102470003F6F3E6B0A0E3C6FD882010EEA6E360E3D
:10248000E96E39C145F138C144F137C143F136C174
:1024900042F141C149F140C148F13FC147F13EC15C
:1024A00046F1000193DF0150005213E101013C515C
:1024B000010AD8A402D000010CD03A510CE00F0B55
:1024C0003C5D01E00FE23ABF0DD03ABD04D0200ED2
:1024D00003D001013A6B300E0026005004009EA884
:1024E000FDD7AD6ED89241C145F140C144F13FC125
:1024F00043F13EC142F1496B486B476B0A0E466F90
:10250000000164DF03C041F102C040F101C03FF1AE
:1025100000C03EF101013C2FAFD70001000CEACF13
:1025200042F1E9CF41F101013B39F0093D6F3D270F
:10253000E20F3E6F320F406F3B510F0B3E273E279D
:102540004027E90F3F6F3F273F273A390F0B3F27BF
:1025500040273F374037401F40373A510F0B402745
:102560003D37070E3C6F0A0E3F074027FDE33E074D
:102570003F27FDE33D073E27FDE33C073D27FDE305
:10258000010EEA6E3C0EE96E070E4115419DE926EB
:10259000400EE95CD8B4418DEF50006E08E141BDBA
:1025A00006D041B90DD041B702D0200E03D04187EB
:1025B0004199300E0026005004009EA8FDD7AD6E54
:1025C000EE5041ADE5D70001000C010E0101375D71
:1025D000F40FD8B0D1D00C0F0001D1EF13F04A0E98
:1025E00004009EA8FDD7AD6E610E04009EA8FDD725
:1025F000AD6E6E0E04009EA8FDD7AD6E0101BCD07D
:10260000460E04009EA8FDD7AD6E650E04009EA880
:10261000FDD7AD6E620E04009EA8FDD7AD6E010120
:10262000ABD04D0E04009EA8FDD7AD6E610E040028
:102630009EA8FDD7AD6E720E04009EA8FDD7AD6EAC
:1026400001019AD0410E04009EA8FDD7AD6E700E18
:1026500004009EA8FDD7AD6E720E04009EA8FDD7A3
:10266000AD6E010189D04D0E04009EA8FDD7AD6E60
:10267000610E04009EA8FDD7AD6E790E04009EA8E1
:10268000FDD7AD6E010178D04A0E04009EA8FDD79B
:10269000AD6E750E04009EA8FDD7AD6E6E0E0400E3
:1026A0009EA8FDD7AD6E010167D04A0E04009EA81A
:1026B000FDD7AD6E750E04009EA8FDD7AD6E6C0EF5
:1026C00004009EA8FDD7AD6E010156D0410E040056
:1026D0009EA8FDD7AD6E750E04009EA8FDD7AD6E09
:1026E000670E04009EA8FDD7AD6E010145D0530EC4
:1026F00004009EA8FDD7AD6E650E04009EA8FDD710
:10270000AD6E700E04009EA8FDD7AD6E010134D0F1
:102710004F0E04009EA8FDD7AD6E630E04009EA868
:10272000FDD7AD6E740E04009EA8FDD7AD6E0101FD
:1027300023D04E0E04009EA8FDD7AD6E6F0E040090
:102740009EA8FDD7AD6E760E04009EA8FDD7AD6E97
:10275000010112D0440E04009EA8FDD7AD6E650E97
:1027600004009EA8FDD7AD6E630E04009EA8FDD7A1
:10277000AD6E010101D00101D00E3625386F070E74
:10278000396FD8B0392B200E04009EA8FDD7AD6E4E
:10279000010EE96E39C13BF138C13AF10001BFDEEB
:1027A000000CE824F76AF736BD0FF66E270EF72205
:1027B0000A00F550FA6E0800F550F96EDE25002685
:1027C0002226442666268826AA26CC26EE26102710
:1027D000322754270900F6CF3AF1F7CF3BF1F550F5
:1027E00004009EA8FDD7AD6E3AC1F6FF3BC1F7FFCE
:1027F0000101392F01D002D00001ECD70001000CFB
:10280000A80EF66E120EF76E040E0101396F00016C
:10281000E1DFC90E04009EA8FDD7AD6E0101326B49
:1028200032513B0807E3CD0E04009EA8FDD7AD6EE4
:10283000322BF6D7BB0E04009EA8FDD7AD6E0D0E51
:1028400004009EA8FDD7AD6E0A0E04009EA8FDD719
:10285000AD6EB00EF66E120EF76E040E396F0001FB
:10286000B9DFBA0E04009EA8FDD7AD6EB60EF66EA7
:10287000120EF76E0D0E0101396F0001ABDF1BA2C6
:102880007CD12550090A15E0050A19E0030A1DE06C
:102890001A0A21E00F0A25E0050A29E03F0A2DE087
:1028A000050A31E0030A35E00E0A39E0610A3DE02D
:1028B00042D0C40EF66E120EF76E56DD42D0DC0E1C
:1028C000F66E120EF76E50DD3CD0F40EF66E120E60
:1028D000F76E4ADD36D00C0EF66E130EF76E44DD41
:1028E00030D0240EF66E130EF76E3EDD2AD03C0E6D
:1028F000F66E130EF76E38DD24D0540EF66E130EFE
:10290000F76E32DD1ED06C0EF66E130EF76E2CDDF8
:1029100018D0840EF66E130EF76E26DD12D09C0EC4
:10292000F66E130EF76E20DD0CD0B40EF66E130E9D
:10293000F76E1ADD06D0CC0EF66E130EF76E14DDB0
:1029400000D025504908D8A481D028500BE0010AB6
:1029500018E0030A25E0010A32E0070A3FE0010A15
:102960004CE05AD0010E0101356F1E0E366F280E55
:10297000376F0001CADC220EF66E0E0EF76EF4DC25
:102980005AD0020E0101356F240E366F280E376FB4
:102990000001BBDCF20EF66E0D0EF76EE5DC4BD0DF
:1029A000020E0101356F230E366F280E376F0001BE
:1029B000ACDC020EF66E0E0EF76ED6DC3CD0010ECD
:1029C0000101356F210E366F280E376F00019DDC37
:1029D000120EF66E0E0EF76EC7DC2DD0010E010141
:1029E000356F240E366F280E376F00018EDC320EE5
:1029F000F66E0E0EF76EB8DC1ED0010E0101356FBB
:102A0000230E366F280E376F00017FDC420EF66E04
:102A10000E0EF76EA9DC0FD0010E0101356F1E0EF0
:102A2000366F2F0E376F000170DC620EF66E0E0EE1
:102A3000F76E9ADC00D0200E04009EA8FDD7AD6E84
:102A4000200E04009EA8FDD7AD6E95D02650010A39
:102A50000DE0030A1AE0010A27E0070A34E0010A40
:102A600041E0030A4EE0090A5CE06BD0020E01016E
:102A7000356F240E366F280E376F000146DCF20EDC
:102A8000F66E0D0EF76E70DC6CD0020E0101356F24
:102A9000230E366F280E376F000137DC020EF66EFC
:102AA0000E0EF76E61DC5DD0010E0101356F210E57
:102AB000366F280E376F000128DC120EF66E0E0EF0
:102AC000F76E52DC4ED0010E0101356F1E0E366FCF
:102AD000280E376F000119DC220EF66E0E0EF76E0F
:102AE00043DC3FD0010E0101356F240E366F280EF6
:102AF000376F00010ADC320EF66E0E0EF76E34DC14
:102B000030D0010E0101356F230E366F280E376F5E
:102B1000000185EC11F0420EF66E0E0EF76E24DC0D
:102B200020D0010E0101356F250E366F280E376F4C
:102B3000000185EC11F0520EF66E0E0EF76E14DCED
:102B400010D0010E0101356F1E0E366F2F0E376F3C
:102B5000000185EC11F0620EF66E0E0EF76E04DCCD
:102B600000D0200E04009EA8FDD7AD6E200E0400FC
:102B70009EA8FDD7AD6E0ADC06D0E40EF66E130EED
:102B8000F76EB4EC11F00C0EF66E140EF76E080E24
:102B90000101396F00011EDEBA0E04009EA8FDD7A8
:102BA000AD6E0D0E04009EA8FDD7AD6E0A0E04009A
:102BB0009EA8FDD7AD6EDA0E04009EA8FDD7AD6EBF
:102BC000C40E04009EA8FDD7AD6EC40E04009EA8DE
:102BD000FDD7AD6EC40E04009EA8FDD7AD6ED00E1D
:102BE00004009EA8FDD7AD6E0101326B32513B0847
:102BF00007E3C40E04009EA8FDD7AD6E322BF6D7B6
:102C0000D00E04009EA8FDD7AD6E326B3251030882
:102C100007E3C40E04009EA8FDD7AD6E322BF6D795
:102C2000BF0E04009EA8FDD7AD6E0D0E04009EA839
:102C3000FDD7AD6E0A0E04009EA8FDD7AD6EB30E93
:102C400004009EA8FDD7AD6EB00EF66E080EF76EAE
:102C5000450E396F0001BEDDB30E04009EA8FDD7FE
:102C6000AD6E0D0E04009EA8FDD7AD6E0A0E0400D9
:102C70009EA8FDD7AD6EB30E04009EA8FDD7AD6E25
:102C8000FC0EF66E080EF76E450E0101396F00015D
:102C9000A1DDB30E04009EA8FDD7AD6E0D0E04009D
:102CA0009EA8FDD7AD6E0A0E04009EA8FDD7AD6E9E
:102CB000B30E04009EA8FDD7AD6E480EF66E090E49
:102CC000F76E450E0101396F000184DDB30E04007B
:102CD0009EA8FDD7AD6E0D0E04009EA8FDD7AD6E6B
:102CE0000A0E04009EA8FDD7AD6EB30E04009EA888
:102CF000FDD7AD6E940EF66E090EF76E450E01010E
:102D0000396F000167DDB30E04009EA8FDD7AD6EDC
:102D10000D0E04009EA8FDD7AD6E0A0E04009EA8FD
:102D2000FDD7AD6E1BA0E9D0B30E04009EA8FDD761
:102D3000AD6EE00EF66E090EF76E450E0101396FAD
:102D4000000148DDB30E04009EA8FDD7AD6E0D0E48
:102D500004009EA8FDD7AD6E0A0E04009EA8FDD704
:102D6000AD6EB30E04009EA8FDD7AD6E2C0EF66EB0
:102D70000A0EF76E450E0101396F00012BDDB30E0F
:102D800004009EA8FDD7AD6E0D0E04009EA8FDD7D1
:102D9000AD6E0A0E04009EA8FDD7AD6EB30E040002
:102DA0009EA8FDD7AD6E780EF66E0A0EF76E450E34
:102DB0000101396F00010EDDB30E04009EA8FDD79E
:102DC000AD6E0D0E04009EA8FDD7AD6E0A0E040078
:102DD0009EA8FDD7AD6EB30E04009EA8FDD7AD6EC4
:102DE000C40EF66E0A0EF76E450E0101396F000132
:102DF000F1DCB30E04009EA8FDD7AD6E0D0E0400ED
:102E00009EA8FDD7AD6E0A0E04009EA8FDD7AD6E3C
:102E1000B30E04009EA8FDD7AD6E100EF66E0B0E1D
:102E2000F76E450E0101396F0001D4DCB30E0400CA
:102E30009EA8FDD7AD6E0D0E04009EA8FDD7AD6E09
:102E40000A0E04009EA8FDD7AD6EB30E04009EA826
:102E5000FDD7AD6E5C0EF66E0B0EF76E450E0101E2
:102E6000396F0001B7DCB30E04009EA8FDD7AD6E2C
:102E70000D0E04009EA8FDD7AD6E0A0E04009EA89C
:102E8000FDD7AD6EB30E04009EA8FDD7AD6EA80EA3
:102E9000F66E0B0EF76E450E0101396F00019ADCDC
:102EA000B30E04009EA8FDD7AD6E0D0E04009EA8C3
:102EB000FDD7AD6E0A0E04009EA8FDD7AD6EB30E11
:102EC00004009EA8FDD7AD6EF40EF66E0B0EF76EE5
:102ED000450E0101396F00017DDCB30E04009EA890
:102EE000FDD7AD6E0D0E04009EA8FDD7AD6E0A0E87
:102EF00004009EA8FDD7AD6E92D0B30E04009EA82C
:102F0000FDD7AD6E400EF66E0C0EF76E450E01014C
:102F1000396F00015FDCB30E04009EA8FDD7AD6ED3
:102F20000D0E04009EA8FDD7AD6E0A0E04009EA8EB
:102F3000FDD7AD6EB30E04009EA8FDD7AD6E8C0E0E
:102F4000F66E0C0EF76E450E0101396F000142DC82
:102F5000B30E04009EA8FDD7AD6E0D0E04009EA812
:102F6000FDD7AD6E0A0E04009EA8FDD7AD6EB30E60
:102F700004009EA8FDD7AD6ED80EF66E0C0EF76E4F
:102F8000450E0101396F000125DCB30E04009EA837
:102F9000FDD7AD6E0D0E04009EA8FDD7AD6E0A0ED6
:102FA00004009EA8FDD7AD6EB30E04009EA8FDD709
:102FB000AD6E240EF66E0D0EF76E450E0101396FE3
:102FC000000108DCB30E04009EA8FDD7AD6E0D0E07
:102FD00004009EA8FDD7AD6E0A0E04009EA8FDD782
:102FE000AD6EB30E04009EA8FDD7AD6E700EF66EEA
:102FF0000D0EF76E450E0101396F0001EAEC13F07A
:10300000B30E04009EA8FDD7AD6E0D0E04009EA861
:10301000FDD7AD6E0A0E04009EA8FDD7AD6EC00EA2
:1030200004009EA8FDD7AD6E0101326B32514408F9
:1030300007E3C40E04009EA8FDD7AD6E322BF6D771
:10304000D90E04009EA8FDD7AD6E0001000C18EC4F
:1030500011F0010E0101356F250E366F280E376F06
:10306000000185EC11F0180EF66E140EF76EB4EC3C
:1030700011F06A0EF66E140EF76EB4EC11F0E20E5B
:10308000F66E0F0EF76EB4EC11F02E0E04009EA833
:10309000FDD7AD6E200E04009EA8FDD7AD6EF60ED6
:1030A000F66E0F0EF76EB4EC11F0760EF66E140E8F
:1030B000F76EB4EC11F0040EF66E100EF76EB4EC71
:1030C00011F02E0E04009EA8FDD7AD6E0D0E04006B
:1030D0009EA8FDD7AD6E0A0E04009EA8FDD7AD6E6A
:1030E0007E0EF66E140EF76EB4EC11F0140EF66E42
:1030F000100EF76EB4EC11F00D0E04009EA8FDD773
:10310000AD6E0A0E04009EA8FDD7AD6E0D0E040034
:103110009EA8FDD7AD6E0A0E04009EA8FDD7AD6E29
:10312000C6EC11F0F2CF32F1F29EAA6A150EA96E2A
:10313000A69CA69EA680A850010132BFF28E1C6EEE
:103140008E0EF66E140EF76E0001B4EC11F0010E47
:103150000101356F250E366F280E376F000185ECA3
:1031600011F0A20EF66E140EF76EB4EC11F01C50B6
:10317000F30F57E20D0FE4EF19F0AA0EF66E140EDE
:10318000F76EB4EC11F04DD0B40EF66E140EF76E6F
:10319000B4EC11F046D0BE0EF66E140EF76EB4EC21
:1031A00011F03FD0C60EF66E140EF76EB4EC11F0AF
:1031B00038D0D20EF66E140EF76EB4EC11F031D09A
:1031C000DE0EF66E140EF76EB4EC11F02AD0EC0E93
:1031D000F66E140EF76EB4EC11F023D0FA0EF66E04
:1031E000140EF76EB4EC11F01CD0060EF66E150E30
:1031F000F76EB4EC11F015D0120EF66E150EF76ED8
:10320000B4EC11F00ED0220EF66E150EF76EB4EC83
:1032100011F007D02E0EF66E150EF76EB4EC11F00D
:1032200000D0200E04009EA8FDD7AD6E2D0E040028
:103230009EA8FDD7AD6E200E04009EA8FDD7AD6EF2
:103240002150DD080EE1225026080BE1235209E14E
:10325000245207E13A0EF66E150EF76EB4EC11F03B
:1032600030D0D89224C045F123C044F122C043F1AC
:1032700021C042F10101496B486B476B0A0E466F52
:103280000001E6EC11F003C035F102C034F101C0D9
:1032900033F100C032F1410EE96E03C039F102C0D2
:1032A00038F101C037F100C036F130EC12F06D0E8C
:1032B00004009EA8FDD7AD6E6C0E04009EA8FDD73D
:1032C000AD6EC6EC11F0420EF66E150EF76EB4EC54
:1032D00011F0C6EC11F0010E0101356F250E366FAD
:1032E000280E376F000185EC11F0F2CF32F1F29E1B
:1032F000AA6A130EA96EA69CA69EA680A8500101DC
:1033000032BFF28E336FF2CF34F1F29EAA6A140EFE
:10331000A96EA69CA69EA680A85034BFF28E356FDB
:1033200033C136F135C137F10001E5EC12F0C6ECDE
:1033300011F0500EF66E150EF76EB4EC11F0010E92
:103340000101356F250E366F280E376F000185ECB1
:1033500011F01AAE10D04F0E04009EA8FDD7AD6E2E
:10336000450E04009EA8FDD7AD6E4D0E04009EA82C
:10337000FDD7AD6E0FD0460E04009EA8FDD7AD6EF2
:10338000540E04009EA8FDD7AD6E200E04009EA82A
:10339000FDD7AD6EC6EC11F00D0E04009EA8FDD752
:1033A000AD6E0A0E04009EA8FDD7AD6E0A0E040095
:1033B0009EA8FDD7AD6E00EC14F05C0EF66E150EF7
:1033C000F76EB4EC11F0000CE824F76AF736E30F5F
:1033D000F66E330EF7220A00F550FA6E0800F5502B
:1033E000F96E7A3188319631A431B231C031CE31A3
:1033F0002232DC31EA31F83106321432010EEA6E43
:10340000390EE96EEF5011E0060E016EBF0E006E30
:103410000400002EFDD7012EF9D77A0E006E002E83
:10342000FED700D00400EF2EEFD7000C93908A90C7
:103430000400030E0101386FF20E396F0001D1EC68
:1034400010F00101382FF8D793800400070E006EAA
:10345000002EFED700D0938081B014D03E0EF66EC1
:10346000100EF76E0001B4EC11F0020E0101386F7E
:10347000FA0E396F0001C2DF0101382FF9D7000EB3
:10348000016E3CD004006B0E006E002EFED700D003
:103490009380379181A037810400EF0E396F0001CE
:1034A000D1EC10F0010137A104D0010E016E26D03D
:1034B00025D06C0EF66E100EF76E0001B4EC11F014
:1034C000020E0101386FFA0E396F000197DF01011A
:1034D000382FF9D79E0EF66E100EF76E0001B4EC81
:1034E00011F0020E0101386FFA0E396F000186DF0C
:1034F0000101382FF9D7000E016E00D00001000C39
:10350000010E0101386F385108082FE393908A901B
:10351000D89037330EE393908A800400200E006E1B
:10352000002EFED700D081B003D0000E016E1FD058
:103530000DD093908A900400200E006E002EFED7CE
:1035400000D081A003D0000E016E11D00400330E14
:10355000006E002EFED793908A800400070E006E46
:10356000002EFED700D0382BCED7010E016E000101
:10357000000C5CDF0152FDE00400020E0101366F19
:10358000D10E396F0001D1EC10F00101362FF8D7C0
:10359000550E376F0001B4DF0400060E006E002EDA
:1035A000FED70101356B3551070821E30400060EF3
:1035B000006E002EFED70001A551080DF350010149
:1035C000376B366F036A35513625016E375103224A
:1035D0000150550FE96E000E0320EA6EEFCF36F171
:1035E00036C137F100018CDF0101352BDCD700013A
:1035F000000C010E0101396F3951080818E393904E
:103600008A9093800400200E006E002EFED700D01A
:10361000938081B002D0D89001D0D8803A33040092
:103620003B0E006E002EFED70000392BE5D73AC1C5
:1036300001F00001000C01013BBF11D00F0E006E24
:103640003A3900160A0E005C03E2300E002602D062
:103650003B510026005004009EA8FDD7AD6E0F0E12
:103660003A170A0E3A5D02E2300E02D03B9F3B5100
:103670003A273A5104009EA8FDD7AD6E0001000C18
:10368000016A026A006A036A01013A5102E1395192
:1036900018E0100E3B6FD8903737383700360336B6
:1036A0003A51035C02E13951005C07E33951005E95
:1036B000D8A003063A51035ED880013602363B2F6C
:1036C000EAD70001000C010137530AE00D0E040097
:1036D0009EA8FDD7AD6E0A0E04009EA8FDD7AD6E64
:1036E000D00EF66E100EF76E0D0E396F0001EAEC7B
:1036F00013F045C03AF1370E01013B6F00019BDF2B
:10370000E00EF66E100EF76E060E0101396F000125
:10371000EAEC13F0010E0101386F3851060817E387
:10372000036A3851450FE96E000E0320EA6EEFCFB1
:1037300039F139C13AF1370E3B6F00017CDF200EC1
:1037400004009EA8FDD7AD6E0101382BE6D7E80E28
:10375000F66E100EF76E060E396F0001EAEC13F0EC
:103760004CC03AF1370E01013B6F000164DF0D0ED2
:1037700004009EA8FDD7AD6E0A0E04009EA8FDD7DA
:10378000AD6E000C53DE0152FDE00400020E01019B
:10379000376FD10E396F0001D1EC10F00101372FD6
:1037A000F8D7330E376F0001ABDE0101366B3651AF
:1037B00007081AE30400060E006E002EFED7036A07
:1037C0003651450F016E000E032201C037F103C0D0
:1037D00038F100010EDF38C1EAFF37C1E9FF01C04F
:1037E000EFFF0101362BE3D7355305E035C137F143
:1037F000000169DF01010001000C0101346B32534B
:1038000021E0000118EC11F0010E0101356F250EC9
:10381000366F280E376F000185EC11F0200EF66E22
:10382000180EF76EB4EC11F0C6EC11F0400EF66E07
:10383000180EF76EB4EC11F0BA0EF66E0D0EF76EB0
:10384000B4EC11F00001A53D01D002D092DE0FD002
:10385000EDDD0152FDE00400DD0E0101396F0001D4
:10386000D1EC10F0CC0E0101376F000149DE0400ED
:10387000A60E006E002EFED7F00E0101376F00017C
:103880003FDE0400A60E006E002EFED70101376B4E
:10389000000136DE0101336B33511F0827E30400BA
:1038A000090E006E002EFED70000036A3351250F6B
:1038B000016E000E032201C035F103C036F1000194
:1038C00098DE36C1EAFF35C1E9FF01C0EFFF010113
:1038D00033511D0809E3036A3351250FE96E000EC9
:1038E0000320EA6EEF503427332BD6D73253D8B4A7
:1038F0009CD2010E356F250E366F280E376F0001F2
:1039000085EC11F00101336B33511F0843E3335150
:103910000F0B29E10001C6EC11F00D0E04009EA86A
:10392000FDD7AD6E0A0E04009EA8FDD7AD6E33C163
:103930003AF1370E01013B6F00017DDE200E0400DD
:103940009EA8FDD7AD6E200E04009EA8FDD7AD6EDB
:10395000010E0101356F250E366F280E376F0001FD
:1039600085EC11F00101036A3351250FE96E000E59
:103970000320EA6EEFCF35F135C13AF1370E3B6FD8
:10398000000159DE200E04009EA8FDD7AD6E010196
:10399000332BBAD70001C6EC11F025504908D8A442
:1039A000C1D028500BE0010A20E0030A35E0010AEB
:1039B0004AE0070A5FE0010A74E08AD0010E0101C3
:1039C000356F1E0E366F280E376F000185EC11F033
:1039D000720EF66E0E0EF76EB4EC11F0220EF66E4D
:1039E0000E0EF76EB4EC11F08AD0020E0101356FA5
:1039F000240E366F280E376F000185EC11F0720E21
:103A0000F66E0E0EF76EB4EC11F0F20EF66E0D0EB1
:103A1000F76EB4EC11F073D0020E0101356F230E76
:103A2000366F280E376F000185EC11F0720EF66EBE
:103A30000E0EF76EB4EC11F0020EF66E0E0EF76E6F
:103A4000B4EC11F05CD0010E0101356F210E366F20
:103A5000280E376F000185EC11F0720EF66E0E0E17
:103A6000F76EB4EC11F0120EF66E0E0EF76EB4ECAB
:103A700011F045D0010E0101356F240E366F280E6E
:103A8000376F000185EC11F0720EF66E0E0EF76EB8
:103A9000B4EC11F0320EF66E0E0EF76EB4EC11F0BF
:103AA0002ED0010E0101356F230E366F280E376FB1
:103AB000000185EC11F0720EF66E0E0EF76EB4EC8E
:103AC00011F0420EF66E0E0EF76EB4EC11F017D038
:103AD000010E0101356F1E0E366F2F0E376F00017C
:103AE00085EC11F0720EF66E0E0EF76EB4EC11F05E
:103AF000620EF66E0E0EF76EB4EC11F000D0C6EC4E
:103B000011F00D0E04009EA8FDD7AD6E0A0E040044
:103B10009EA8FDD7AD6E0A0E04009EA8FDD7AD6E1F
:103B200084D1EDD0200E04009EA8FDD7AD6E2650A6
:103B3000010A0DE0030A1CE0010A2BE0070A3AE043
:103B4000010A49E0030A58E0090A67E077D0020E4B
:103B50000101356F240E366F280E376F000185EC9A
:103B600011F0F20EF66E0D0EF76EB4EC11F077D088
:103B7000020E0101356F230E366F280E376F0001DC
:103B800085EC11F0020EF66E0E0EF76EB4EC11F02D
:103B900066D0010E0101356F210E366F280E376F8A
:103BA000000185EC11F0120EF66E0E0EF76EB4ECFD
:103BB00011F055D0010E0101356F1E0E366F280E23
:103BC000376F000185EC11F0220EF66E0E0EF76EC7
:103BD000B4EC11F044D0010E0101356F240E366FA4
:103BE000280E376F000185EC11F0320EF66E0E0EC6
:103BF000F76EB4EC11F033D0010E0101356F230ED6
:103C0000366F280E376F000185EC11F0420EF66E0C
:103C10000E0EF76EB4EC11F022D0010E0101356FDB
:103C20000F0E366F280E376F000185EC11F0520E23
:103C3000F66E0E0EF76EB4EC11F011D0010E01010C
:103C4000356F1E0E366F2F0E376F000185EC11F0A9
:103C5000620EF66E0E0EF76EB4EC11F000D0C6ECEC
:103C600011F0600EF66E180EF76EB4EC11F0010E46
:103C70000101356F250E366F280E376F000185EC78
:103C800011F041C036F142C035F141C038F142C0B7
:103C900037F101013A6B0A0E396F0001F1DC02C005
:103CA00036F101C035F1000EE96E02C03BF101C0F2
:103CB0003AF18FEC12F06D0E04009EA8FDD7AD6EA8
:103CC0006C0E04009EA8FDD7AD6EC6EC11F0720E0E
:103CD000F66E180EF76EB4EC11F0010E0101356F9F
:103CE000250E366F280E376F000185EC11F031C0BC
:103CF00036F132C037F1E5EC12F0C6EC11F0FF0EF0
:103D0000D88001013455445CD8B480D01EC035F150
:103D1000366B1E504908D8A479D03653D8A476D033
:103D2000FF0ED8803455356F840EF66E180EF76E80
:103D3000120E396F0001EAEC13F044C03AF1370E6D
:103D400001013B6F000177DC200E04009EA8FDD727
:103D5000AD6E35C13AF1370E01013B6F00016BDCEE
:103D6000FF0ED88001013455446E356B00010ADD29
:103D700016EC1AF00152FCE0990E0101376F0001B8
:103D800080EC1AF00400F90E0101396F0001D1EC4A
:103D900010F00101336B33511F0811E3036A3351F3
:103DA000250FE96E000E0320EA6EEFCF35F135C125
:103DB00037F1000180EC1AF00101332BECD7336BA3
:103DC0003351070811E3036A3351450FE96E000EC2
:103DD0000320EA6EEFCF35F135C137F1000180ECF9
:103DE0001AF00101332BECD79E0EF66E180EF76E0B
:103DF0000001B4EC11F0020E0101356F960E396F1F
:103E00000001FEEC19F00101352FF8D70D0E04006A
:103E10009EA8FDD7AD6E0A0E04009EA8FDD7AD6E1C
:103E20000A0E04009EA8FDD7AD6E0001000C040030
:103E3000E2EF10F0015212E104001E6A1D6A1B92AB
:103E40001F501D5C03E120501E5C06E027EC18F0BB
:103E50001EC020F01DC01FF020D01FD01BB204D008
:103E60000101326B0001C9DC1B822550490805E1C4
:103E700025C01EF028C01DF004D025C01EF026C0AD
:103E80001DF01F501D5C03E120501E5C06E01EC0AB
:103E900020F01DC01FF027EC18F0F29430EF04F072
:103EA0000A0D43757272656E74204372656469749D
:103EB0007320636F756E743A20256C750A0D0000CF
:103EC00092908990000C9280000C1B0E04009EA81A
:103ED000FDD7AD6E630E04009EA8FDD7AD6E9DEFBD
:103EE00051F0196AF2BE198EF29E020E0101356F71
:103EF000250E366F280E376F000185EC11F019BEC4
:103F0000F28EBE6BBE5118080DE3BF6BBF514F0858
:103F100007E3200E04009EA8FDD7AD6EBF2BF6D799
:103F2000BE2BF0D7196AF2BE198EF29EC6EC11F0C4
:103F300019BEF28E9FEF51F0F2CF02F1F29EAA6A03
:103F4000100EA96EA69CA69EA680A850010102BFD5
:103F5000F28E036FF2CF04F1F29EAA6A110EA96EDF
:103F6000A69CA69EA680A85004BFF28E056F03C132
:103F7000FDF005C1FCF00001FD51260838E2FF0A02
:103F800003E1FC51100833E2FD6B320EFC6FFDC003
:103F900002F10101036BAA6A100EA96E02C1A8FF0B
:103FA000A69CA69EA684F250006EF29E0F01550EAE
:103FB000A76EAA0EA76EA682A6B2FED7A694005040
:103FC000F212AA6A110EA96EFCC0A8FFA69CA69EBA
:103FD000A684F2CF00F0F29E550EA76EAA0EA76E31
:103FE000A682A6B2FED7A6940050F2120001FC539E
:103FF00024E1FD5322E1740EF66E170EF76E196A76
:10400000F2BE198EF29EB4EC11F019BEF28E080EBB
:104010000101026F196AF2BE198EF29EFA0E396F13
:104020000001FEEC19F019BEF28E0101022FF2D749
:10403000000E016EC6D0C5D00001FD5371E1FC51E8
:1040400031086EE3AC0EF66E170EF76E196AF2BE0B
:10405000198EF29E170E0101396F0001EAEC13F080
:1040600019BEF28E100EE96E196AF2BE198EF29E1A
:10407000FDC03BF1FCC03AF18FEC12F019BEF28E9C
:10408000C60EF66E170EF76E196AF2BE198EF29E04
:10409000070E0101396F0001EAEC13F019BEF28E30
:1040A000FD5303E1FC51010805E2730E04009EA8D4
:1040B000FDD7AD6ECE0EF66E170EF76E196AF2BE14
:1040C000198EF29EB4EC11F019BEF28EE20EF66E6D
:1040D0000F0EF76E196AF2BE198EF29EB4EC11F053
:1040E00019BEF28EF40EF66E170EF76E196AF2BE56
:1040F000198EF29EB4EC11F019BEF28E080E010179
:10410000026F196AF2BE198EF29EFA0E396F000123
:10411000FEEC19F019BEF28E0101022FF2D7000158
:10412000F2CF02F1F29EAA6A160EA96EA69CA69E76
:10413000A680A850010102BFF28E036FF2CF04F1F6
:10414000F29EAA6A170EA96EA69CA69EA680A850EB
:1041500004BFF28E056FF2CF06F1F29EAA6A180E26
:10416000A96EA69CA69EA680A85006BFF28E076FD9
:10417000016B03C100F105C1FFF007C1FEF00001B2
:10418000FE51DD081AE1FF51260817E10101005335
:10419000D8B402D0000111D00153D8B402D000012C
:1041A0000CD00001FD5309E1FC511D0806E3000E8F
:1041B000016E010106D005D00001010E016E010162
:1041C00000D00001B1EF2AF0FC51FE03F3CF01F063
:1041D000F4CF00F0FF03F3500026FD51FE03F3502F
:1041E0000020026E000C8E0E006EFDC001F0FCC0BF
:1041F00002F0036A015209E102C001F0026A080EEE
:10420000005E015202E1006A08D0D89001BE04D0DD
:10421000023601360006F9D7019E000CB60E006E7C
:10422000036A026A016AFC51FD11FE11FF1102E1ED
:10423000006A0DD0D89001BE09D0FC37FD37FE379B
:10424000FF37033602360136002EF4D7019EF6EF13
:1042500031F0FC51D8B4B4D00101086F0051D8A49A
:1042600002D00001ADD0085F07E37F0E0827D8A079
:1042700002D00001A5D00AD0810E085FD8B002D0CC
:1042800000019ED0D8A402D000019AD008C100F04D
:10429000016A026A036A076BFDC006F1068FFEC061
:1042A00005F1FFC004F1190E086F0351045F0DE220
:1042B000010E055F0AE2065F08E2075F06E2072BD0
:1042C000062B052B0351042728D00251055F12E26B
:1042D000010E065F0FE2075F0DE2072B062B02516E
:1042E00005270351042719E3052B17E1062B15E1D8
:1042F000072B13D001518009065F0EE2010E075F04
:104300000BE2072B01518009062702510527E9E33B
:10431000062BE7E1072BE5D70380082F01D00BD050
:10432000D8900437053706370737D890033602365A
:1043300001360937BAD709A106D0D8900132023226
:104340000332093304D0002E02D0000139D009BF56
:104350001ED0D89004370537063707370351045F5E
:1043600007E2010E055F04E2065F02E2075F1DE35C
:104370000251055F05E2010E065F02E2075F15E3E9
:1043800001518009065F03E2010E075F0EE3032A75
:104390000CE1022A0AE1012A08E1002AD8A402D08D
:1043A00000010ED0013202320332FDC008F101518A
:1043B000081B08AF02D0018E08D0019E06D0000174
:1043C000006A016A026A036A0101000116EF32F015
:1043D000800ED8A202D00101051B01010A6B0B6BF4
:1043E00001C109F10551091B0051D8B4DFD0086F94
:1043F000006E0451D8B4E3D0085FD8B483D03EE354
:1044000005C10EF10E8F06C10DF107C10CF10B6B4A
:10441000D8900E330D330C330B33082FF8D709AF78
:1044200003D00A81E0D00A9108910A89010EEA6E50
:10443000030EE96EEBD00A9909BF0AD008A113D088
:104440000E330D330C330B33002AD8B4C7D00BD046
:104450000EBF0CD0D8900B370C370D370E37000637
:10446000D8B4BCD0F5D70A8D6DD00A9D01C109F131
:1044700001AF02D00E8FABD00E9FA9D004C108F1BE
:1044800004C100F00051085F01C10EF10E8F02C19E
:104490000DF103C10CF10B6BD8900E330D330C33BF
:1044A0000B33082FF8D709AF03D00A839CD00A93A7
:1044B00008910A8B010EEA6E070EE96EA7D00A9BDF
:1044C00009BF0AD008A113D00E330D330C330B33C0
:1044D000002AD8B483D00BD00EBF0CD0D8900B37A5
:1044E0000C370D370E370006D8B478D0F5D70A8FC1
:1044F00029D00A9F05C109F105AF02D00E8F67D000
:104500000E9F65D005C10EF10E8F06C10DF107C1DA
:104510000CF109AF04D00E9F0A8565D00A950B6B8C
:104520000891010EEA6E030EE96E70D009BF1CD02F
:1045300001C109F108A106D00E330D330C330B3342
:10454000002A4CE00BAF0BD00C2B09E10D2B07E13F
:104550000E2B05E10E330D330C33002A3FE00ABD6C
:1045600084D70ABFC6D71CD0800E0E1B0EAF04D056
:104570003AD005C109F10AD001C109F10E5306E193
:104580000D5304E10C5302E1006A21D00EBF08D0A4
:10459000D8900B370C370D370E37002EF7D71ED0BB
:1045A00009AF02D00E8F13D00E9F11D004C100F0BE
:1045B00005C10EF106C10DF107C10CF108D000C113
:1045C00000F001C10EF102C10DF103C10CF10EC1E9
:1045D00001F00DC102F00CC103F034D0006A016A91
:1045E000026A036A2FD00B6B0C1F0D1F0E1F0B1FCF
:1045F0000B2B05E10C2B03E10D2B01E10E2B0AB176
:1046000012D70AB354D70AB589D7B3D7EF500C27BE
:1046100005E30D2B03E10E2BD8B40881ED52EF50CA
:104620000D2703E30E2BD8B40881ED52EF50EFBEF7
:1046300001D0800A0E27D8B008810AB9FCD60ABB7F
:104640003ED774D7000130EF32F00101016B026BED
:10465000036B0C0E0001FC250101046F000E00012C
:10466000FD210101056F05C103F00451E96E03C08E
:10467000EAFFF2CF08F1F29EAA6A130EA96EA69C79
:10468000A69EA680A85008BFF28EEF6E0D0E000108
:10469000FC250101046F000E0001FD210101056FE1
:1046A00005C103F00451E96E03C0EAFFF2CF08F13F
:1046B000F29EAA6A140EA96EA69CA69EA680A85079
:1046C00008BFF28EEF6E1ABE17D12150DD08D8A4B4
:1046D000A1D022502608D8A49DD02352D8A49AD085
:1046E0002452D8A497D00C0E0001FC250101046FC0
:1046F000000E0001FD210101056F04C1E9FF05C1A4
:10470000EAFF140EEF6E0D0E0001FC250101046F8F
:10471000000E0001FD210101056F04C1E9FF05C183
:10472000EAFF080EEF6E210E0001FC250101046F67
:10473000000E0001FD210101056F0001FE51F00F87
:1047400050E2100F11EF25F005C103F0010104C183
:10475000E9FF05C1EAFF010EEF6E000142D005C17D
:1047600003F0010104C1E9FF05C1EAFF020EEF6E8B
:10477000000137D005C103F0010104C1E9FF05C103
:10478000EAFF030EEF6E00012CD005C103F001011A
:1047900004C1E9FF05C1EAFF040EEF6E000121D05C
:1047A00005C103F0010104C1E9FF05C1EAFF050EDF
:1047B000EF6E000116D005C103F0010104C1E9FF4D
:1047C00005C1EAFF060EEF6E00010BD005C103F034
:1047D000010104C1E9FF05C1EAFF070EEF6E000108
:1047E00000D0020EFF6FFF51040812E3200EFF25D8
:1047F000FC250101046F000E0001FD210101056F80
:1048000004C1E9FF05C1EAFFEF6A0001FF2BEBD706
:1048100027D00101010E0001FF6FFF51040820E3C2
:10482000200EFF25FC250101046F000E0001FD2173
:104830000101056F05C103F00451E96E03C0EAFFF1
:10484000F2CF08F1F29EAA6AFFC0A9FFA69CA69E1D
:10485000A680A85008BFF28EEF6E0001FF2BDDD7B7
:10486000200EFC250101046F000E0001FD21010155
:10487000056F0001FF6BFF5106082EE30101006B7D
:104880000051070823E3000E02B1010E066F05C1B7
:1048900003F004C1E9FF05C1EAFFEFCF07F107C14B
:1048A00000F00051016E04E0D8900032012EFCD7D8
:1048B000000E00B0010E061905E0D89002338C0EF0
:1048C000021B02D0D8900233002BDAD7042BD8B4C5
:1048D000052B0001FF2BCFD7270EFC250101046F0C
:1048E000000E0001FD210101056F04C1E9FF05C1B2
:1048F000EAFF02C1EFFF2ED0196AF2BE198EF29EB6
:10490000356B0001C2EC1BF019BEF28EFF6BFF513C
:10491000070820E3200EFF25FC250101046F000E8F
:104920000001FD210101056F05C103F0036A0001CB
:10493000FF51450FE96E000E0320EA6EEFCF08F13C
:10494000010105C1EAFF04C1E9FF08C1EFFF000151
:10495000FF2BDDD70001FF6BFF511D0812E3FF5154
:10496000FC250101046F000E0001FD210101056F0E
:1049700004C1E9FF05C1EAFFEF5001270001FF2B49
:10498000EBD71E0EFC250101046F000E0001FD2176
:104990000101056F04C1E9FF05C1EAFF01C1EFFF95
:1049A000100E0001FF6FFF51130812E3FF51FC25A9
:1049B0000101046F000E0001FD210101056F04C11A
:1049C000E9FF05C1EAFFEF5003270001FF2BEBD7FA
:1049D000200EFF6FFF51270812E3FF51FC25010154
:1049E000046F000E0001FD210101056F04C1E9FF04
:1049F00005C1EAFFEF5003270001FF2BEBD71F0E85
:104A0000FC250101046F000E0001FD210101056F6D
:104A100004C1E9FF05C1EAFF03C1EFFF000145EF53
:104A200032F0E824F76AF7363D0FF66E4A0EF722A9
:104A30000A00F550FA6E0800F550F96E48475E47D7
:104A400074478A47A047B647E247E247E247E24752
:104A5000E247E247E247E247E247CC471B0E040049
:104A60009EA8FDD7AD6E5B0E04009EA8FDD7AD6E6F
:104A7000730E04009EA8FDD7AD6E000C1B0E040043
:104A80009EA8FDD7AD6E5B0E04009EA8FDD7AD6E4F
:104A9000750E04009EA8FDD7AD6E000C0101006BE1
:104AA0000001FF6BFE5302E018EC11F0F2CF01F1B0
:104AB000F29EAA6A100EA96EA69CA69EA680A85079
:104AC000010101BFF28E026FF2CF03F1F29EAA6ADA
:104AD000110EA96EA69CA69EA680A85003BFF28EBA
:104AE000046F02C100F104C1FFF0005126083DE24D
:104AF000FF0A08E10001FF511008D8A002D001010F
:104B000034D00101006B320E0001FF6F00C101F1D2
:104B10000101026BAA6A100EA96E01C1A8FFA69C32
:104B2000A69EA684F250006EF29E0F01550EA76E4F
:104B3000AA0EA76EA682A6B2FED7A6940050F212C5
:104B4000AA6A110EA96EFFC0A8FFA69CA69EA68405
:104B5000F2CF00F0F29E550EA76EAA0EA76EA682A7
:104B6000A6B2FED7A6940050F2120001FC51FF5FDE
:104B7000000E0101005B00C101F1026BAA6A100E78
:104B8000A96E01C1A8FFA69CA69EA684F250006E45
:104B9000F29E0F01550EA76EAA0EA76EA682A6B2B0
:104BA000FED7A6940050F212AA6A110EA96EFFC099
:104BB000A8FFA69CA69EA684F2CF00F0F29E550EFA
:104BC000A76EAA0EA76EA682A6B2FED7A694005024
:104BD000F212060EF66E170EF76E196AF2BE198EF5
:104BE000F29E0001B4EC11F019BEF28EFD530DE1FE
:104BF0000C0EF66E170EF76E196AF2BE198EF29E43
:104C0000B4EC11F019BEF28E0CD0160EF66E170E23
:104C1000F76E196AF2BE198EF29EB4EC11F019BE4D
:104C2000F28E320EF66E170EF76E196AF2BE198EFC
:104C3000F29EB4EC11F019BEF28E4C0EF66E170E09
:104C4000F76E196AF2BE198EF29E210E0101396FBC
:104C50000001EAEC13F019BEF28E100EE96E196A2B
:104C6000F2BE198EF29E00C13BF1FFC03AF18FEC0B
:104C700012F019BEF28E0A0E04009EA8FDD7AD6E8A
:104C80000D0E04009EA8FDD7AD6E080E0101016F48
:104C9000196AF2BE198EF29EFA0E396F0001FEEC0F
:104CA00019F019BEF28E0101012FF2D70001000C9C
:104CB0008E0E006EFC51005EFDC002F0FEC001F0E1
:104CC000028E005209E0D890025202E1015204E043
:104CD00002320132002EF7D7FDAF05D0011E021EB1
:104CE000012AD8B4022A000C04009EA8FDD7AD6E9C
:104CF000000C04009EAAFDD7AECF05F101010551BD
:104D00000001F2DF01010551390805E3300E055DB0
:104D1000016E0FD00ED00551600806E205517A08E9
:104D200003E30551DF0B01D00551BF0F0A0F016EE0
:104D300000D00001000CDDDF01C004F1DADF01C0AA
:104D400003F101010351DD0804E104C101F007D0C2
:104D500006D00451100DF3500325016E00D0000160
:104D6000000C010109070A6B04009EAAFDD7AECF13
:104D70000BF10B5108080EE10A530BE00A070B5127
:104D80000001B2DF200EB0DF01010B510001ACDFEA
:104D9000010117D00B511F0814E20B517E0811E3DB
:104DA0000A51095D0EE30A510A2B036A0725E96ED1
:104DB00008510320EA6E0BC1EFFF0B51000194DF95
:104DC00001010B510D08D0E1036A0A510725E96E74
:104DD00008510320EA6EEF6A0001000C006A016AC4
:104DE00001010E51D8900FB10026003201320FB3ED
:104DF0000026003201320FB50026003201320FB713
:104E00000026003201320FB90026003201320FBBFA
:104E10000026003201320FBD0026003201320FBFE2
:104E2000002600320132000184EF27F001010C6BF3
:104E30000A6B0A0E0B6F096B0751081103E1000E94
:104E4000016EC3D00C510C2B036A0725E96E085183
:104E50000320EA6EEFCF0DF10D512D080DE1010E8B
:104E60000A6F0C510C2B036A0725E96E08510320C9
:104E7000EA6EEFCF0DF10DD00D512B080AE10C5168
:104E80000C2B036A0725E96E08510320EA6EEFCF69
:104E90000DF10D512F08D8B090D00D513908D8A080
:104EA0008CD00D51300821E1036A0C510725E96EC1
:104EB00008510320EA6EEF5078080AE0036A0C51AB
:104EC0000725E96E08510320EA6EEF5058080DE1FE
:104ED000100E0B6F0C2B0C510C2B036A0725E96E7F
:104EE00008510320EA6EEFCF0DF10B510A081DE1C6
:104EF0000D512F0819E20D51390816E30A0E0E6FF5
:104F000009C10FF100016AD7300E01010D5D0124C6
:104F1000096F0C510C2B036A0725E96E0851032019
:104F2000EA6EEFCF0DF1E4D748D00B51100845E100
:104F30000D51600806E20D517A0803E30D51DF0BB5
:104F400001D00D510D6F0D512F0803E20D5139089D
:104F500006E20D51400831E20D5146082EE30D5195
:104F60002F080CE20D51390809E309390E6FF00ED4
:104F70000E17300E0D5D0E25096F09D009390E6F21
:104F8000F00E0E17410E0D5D0A0F0E25096F0C5124
:104F90000C2B036A0725E96E08510320EA6EEFCF58
:104FA0000DF10D51600806E20D517A0803E30D5131
:104FB000DF0B01D00D510D6FC6D70A2D04D00B5158
:104FC0000A0801E1096D09C101F00001F6EF27F0BF
:104FD000010E0101086F076F050E096F0001C1DEA8
:104FE000010E0101086F076F000120D701C006F113
:104FF000010106C101F00001000CFC53D8B473D0CC
:10500000AA0EF66E180EF76E196AF2BE198EF29E8F
:10501000B4EC11F019BEF28E8EDE01C0FDF0FD5130
:105020001F0801E2EDD7CA0EF66E180EF76E196A68
:10503000F2BE198EF29EB4EC11F019BEF28EC8DFEA
:1050400001C000F1FD5101010027FDC0FFF000513A
:105050000001FF5D47E2FF511F0B0101016FE80EE8
:10506000F66E180EF76E196AF2BE198EF29E1E0EBB
:10507000396F0001EAEC13F019BEF28E196AF2BE24
:10508000198EF29E01C13AF1370E01013B6F00010A
:105090001BEC1BF019BEF28E3A0E04009EA8FDD741
:1050A000AD6E2D0E04009EA8FDD7AD6E200E04003F
:1050B0009EA8FDD7AD6EFF511F0B036A250F016E31
:1050C000000E032201C001F103C002F1000133DE32
:1050D00002C1EAFF01C1E9FF01C0EFFFFF2B01019F
:1050E000B6D7000105D0FE51FD250101006F00017A
:1050F000A53D01D009D0196AF2BE198EF29EB9EC15
:105100001AF019BEF28E23D0196AF2BE198EF29EE1
:1051100016EC1AF019BEF28E0152F6E00400196A7C
:10512000F2BE198EF29EDD0E0101396F0001D1EC45
:1051300010F019BEF28E196AF2BE198EF29ECC0ED4
:105140000101376F000180EC1AF019BEF28E0400E5
:10515000090E006E002EFED70000196AF2BE198EED
:10516000F29E0F0E0101376F000180EC1AF019BE9C
:10517000F28E0400090E006E002EFED70000196AA0
:10518000F2BE198EF29EFDC037F180EC1AF019BE06
:10519000F28EFDC0FFF0010100510001FF5D1BE236
:1051A0000400090E006E002EFED70000036AFF51B6
:1051B000250FE96E000E0320EA6EEFCF01F1196AA8
:1051C000F2BE198EF29E01C137F180EC1AF019BEC1
:1051D000F28EFF2BE0D7FC530FE00D0E04009EA8CB
:1051E000FDD7AD6E0A0E04009EA8FDD7AD6E0A0E67
:1051F00004009EA8FDD7AD6E000CFC530CE0BA0E67
:10520000F66E0D0EF76E196AF2BE198EF29EB4ECB0
:1052100011F019BEF28EA53D01D009D0196AF2BE77
:10522000198EF29EB9EC1AF019BEF28E23D0196ACB
:10523000F2BE198EF29E16EC1AF019BEF28E0152D1
:10524000F6E00400196AF2BE198EF29EDD0E01012D
:10525000396F0001D1EC10F019BEF28E196AF2BE5E
:10526000198EF29ECC0E0101376F000180EC1AF00E
:1052700019BEF28E0400090E006E002EFED700004B
:10528000196AF2BE198EF29EAA0E0101376F000153
:1052900080EC1AF019BEF28E0400090E006E002E8A
:1052A000FED70000196AF2BE198EF29E0101376B1B
:1052B000000180EC1AF019BEF28EFD6BFD511F0843
:1052C00022E30400090E006E002EFED70000036AE0
:1052D000FD51FE0F016E000E032201C01EF10101FF
:1052E00003C01FF1196AF2BE198EF29E0001F9EC9B
:1052F0001AF019BEF28E1FC1EAFF1EC1E9FF01C0FC
:10530000EFFFFD2BDBD7FC53D8B473D0FD6BFD5101
:105310001F0860E3FD510F0B3FE1036AFD51FE0FD3
:10532000E96E000E0320EA6EEFCF1EF10D0E0400B1
:105330009EA8FDD7AD6E0A0E04009EA8FDD7AD6EE7
:10534000196AF2BE198EF29EFDC03AF1370E0101C4
:105350003B6F00011BEC1BF019BEF28E200E040007
:105360009EA8FDD7AD6E200E04009EA8FDD7AD6EA1
:10537000196AF2BE198EF29E1EC13AF1370E010172
:105380003B6F00011BEC1BF019BEF28E200E0400D7
:105390009EA8FDD7AD6E1CD0036AFD51FE0FE96ECD
:1053A000000E0320EA6EEFCF1EF1196AF2BE198ECD
:1053B000F29E1EC13AF1370E01013B6F00011BEC5A
:1053C0001BF019BEF28E200E04009EA8FDD7AD6E14
:1053D000FD2B9DD70D0E04009EA8FDD7AD6E0A0EC5
:1053E00004009EA8FDD7AD6E0A0E04009EA8FDD74E
:1053F000AD6E000CA53D01D009D0196AF2BE198E20
:10540000F29EB9EC1AF019BEF28E23D0196AF2BEE0
:10541000198EF29E16EC1AF019BEF28E0152F6E0C9
:105420000400196AF2BE198EF29EDD0E0101396F79
:105430000001D1EC10F019BEF28E196AF2BE198E7D
:10544000F29ECC0E0101376F000180EC1AF019BEFC
:10545000F28E0400090E006E002EFED70000196ABD
:10546000F2BE198EF29E550E0101376F000180ECDD
:105470001AF019BEF28E0400090E006E002EFED73F
:105480000000196AF2BE198EF29EA50E0101376F57
:10549000000180EC1AF019BEF28E196AF2BE198E64
:1054A000F29E060E0101396F0001FEEC19F019BEE3
:1054B000F28E0E0EF66E190EF76E196AF2BE198E86
:1054C000F29EB4EC11F019BEF28E196AF2BE198E7A
:1054D000F29E0A0E0101396F0001FEEC19F019BEAF
:1054E000F28E000CBF6BC06B0A0EC16F020EC26F52
:1054F000420EC36F310EC46F380EC56FC66F340EC7
:10550000C76F390EC86F350EC96F200ECA6FCB6BCF
:10551000CC6BCD6BCE6BCF6BD06BD16BD26BD36BB7
:10552000D46BD56BD66BD76FD86FD96BDA6BDB6B5F
:10553000DC6BDD6BDE6B140EDF6FE06BE16BE26B3F
:10554000E36BE46BE56BE66B550EE76FE86FE96FB5
:10555000EA6FEB6FEC6FED6FEE6F18EC11F09CEFF4
:105560001FF001521EE1F80EF66E1B0EF76E196A5F
:10557000F2BE198EF29EB4EC11F019BEF28E080E36
:10558000FC6F196AF2BE198EF29EFA0E0101396F94
:105590000001FEEC19F019BEF28EFC2FF2D79CEF41
:1055A00034F01C50F30FD8B01FEF31F00D0F9DEF0A
:1055B00034F00C0EBF6F070EC16F010EC26F300EBC
:1055C000C36F340EC46F300EC56F380EC66F330E06
:1055D000C76F310EC86F300EC96FD892196AF2BE0C
:1055E000198EF29E24C045F123C044F122C043F13C
:1055F00021C042F10101496B486B476B0A0E466FAF
:105600000001E6EC11F019BEF28E03C0FFF002C0FB
:10561000FEF001C0FDF00050FC6FDC0806E1FD5318
:1056200004E1FE5302E1FF5328E0D892196AF2BE6A
:10563000198EF29E24C045F123C044F122C043F1EB
:1056400021C042F10101496B486B476B0A0E466F5E
:105650000001E6EC11F019BEF28E03C0FFF002C0AB
:10566000FEF001C0FDF00050FC6FB8083BE1FD2DDD
:1056700039D0FE5337E1FF5335E1D892196AF2BEB3
:10568000198EF29E24C045F123C044F122C043F19B
:1056900021C042F10101496B486B476B0A0E466F0E
:1056A0000001E6EC11F019BEF28E01C0CDF0D892E7
:1056B000196AF2BE198EF29E24C045F123C044F14E
:1056C00022C043F121C042F10101496B486B476B95
:1056D0000A0E466F0001E6EC11F019BEF28E00C012
:1056E000CEF004D0010ECD6FB80ECE6F030ECF6F8B
:1056F000750ED06FC30ED16F540ED26F040ED36FE0
:105700001FEF31F00F0EBF6F070EC16F010EC26F9A
:10571000350EC36F360EC46F310EC56FC66FC76FBF
:10572000C86F370EC96FD892196AF2BE198EF29EF1
:1057300024C045F123C044F122C043F121C042F10D
:105740000101496B486B476B0A0E466F0001E6EC9E
:1057500011F019BEF28E03C0FFF002C0FEF001C0CE
:10576000FDF00050FC6FDC0806E1FD5304E1FE5340
:1057700002E1FF5328E0D892196AF2BE198EF29E18
:1057800024C045F123C044F122C043F121C042F1BD
:105790000101496B486B476B0A0E466F0001E6EC4E
:1057A00011F019BEF28E03C0FFF002C0FEF001C07E
:1057B000FDF00050FC6FB8083BE1FD2D39D0FE53E1
:1057C00037E1FF5335E1D892196AF2BE198EF29E85
:1057D00024C045F123C044F122C043F121C042F16D
:1057E0000101496B486B476B0A0E466F0001E6ECFE
:1057F00011F019BEF28E01C0CDF0D892196AF2BE36
:10580000198EF29E24C045F123C044F122C043F119
:1058100021C042F10101496B486B476B0A0E466F8C
:105820000001E6EC11F019BEF28E00C0CEF004D0FB
:10583000010ECD6FB80ECE6F030ECF6F960ED06FE8
:105840009C0ED16F740ED26F2E0ED36F1FEF31F0FE
:105850001A0EBF6F0A0EC16F020EC26F480EC36FE1
:10586000320EC46F390EC56F360EC66F310EC76F5C
:10587000340EC86F330EC96F030ECF6FD892196AFA
:10588000F2BE198EF29E24C045F123C044F122C01D
:1058900043F121C042F10101496B486B476B0A0E8D
:1058A000466F0001E6EC11F019BEF28E03C0FFF066
:1058B00002C0FEF001C0FDF00050FC6FB80806E128
:1058C000FD2D04D0FE5302E1FF5329E0D892196A5E
:1058D000F2BE198EF29E24C045F123C044F122C0CD
:1058E00043F121C042F10101496B486B476B0A0E3D
:1058F000466F0001E6EC11F019BEF28E03C0FFF016
:1059000002C0FEF001C0FDF00050FC6FD0083CE189
:10591000FD51070839E1FE5337E1FF5335E1D892D5
:10592000196AF2BE198EF29E24C045F123C044F1DB
:1059300022C043F121C042F10101496B486B476B22
:105940000A0E466F0001E6EC11F019BEF28E01C09E
:10595000CDF0D892196AF2BE198EF29E24C045F19C
:1059600023C044F122C043F121C042F10101496B3F
:10597000486B476B0A0E466F0001E6EC11F019BE4A
:10598000F28E00C0CEF004D0010ECD6FB80ECE6FF7
:10599000A10ED06F470ED16FFA0ED26F2B0ED36FC0
:1059A00024520AE1235208E1225010081FE2FF0AA4
:1059B00003E1215030081AE2440EC26F200EC36F7B
:1059C000430EC46F300EC56F340EC66F300EC76FF6
:1059D000330EC86F390EC96F050ECF6FFA0ED06F38
:1059E000830ED16F690ED26F350ED36F1FEF31F07A
:1059F000200EBF6F070EC16F410EC26F200EC36F26
:105A0000300EC46F580EC56F450EC66F340EC76F8B
:105A1000330EC86F310EC96FD892196AF2BE198E53
:105A2000F29E24C045F123C044F122C043F121C0BD
:105A300042F10101496B486B476B0A0E466F00014A
:105A4000E6EC11F019BEF28E03C0FFF002C0FEF0CA
:105A500001C0FDF00050FC6FB80806E1FD2D04D038
:105A6000FE5302E1FF5329E0D892196AF2BE198E63
:105A7000F29E24C045F123C044F122C043F121C06D
:105A800042F10101496B486B476B0A0E466F0001FA
:105A9000E6EC11F019BEF28E03C0FFF002C0FEF07A
:105AA00001C0FDF00050FC6FD0083CE1FD5107083B
:105AB00039E1FE5337E1FF5335E1D892196AF2BE5E
:105AC000198EF29E24C045F123C044F122C043F157
:105AD00021C042F10101496B486B476B0A0E466FCA
:105AE0000001E6EC11F019BEF28E01C0CDF0D892A3
:105AF000196AF2BE198EF29E24C045F123C044F10A
:105B000022C043F121C042F10101496B486B476B50
:105B10000A0E466F0001E6EC11F019BEF28E00C0CD
:105B2000CEF004D0010ECD6FB80ECE6F060ECF6F43
:105B3000050ED06F400ED16FDF0ED26F6F0ED36F98
:105B40007ED3250EBF6F0D0EC16F410EC26F200EAA
:105B5000C36F430EC46F390EC56F380EC66F340E57
:105B6000C76F390EC86F350EC96FD892196AF2BE69
:105B7000198EF29E24C045F123C044F122C043F1A6
:105B800021C042F10101496B486B476B0A0E466F19
:105B90000001E6EC11F019BEF28E03C0FFF002C066
:105BA000FEF001C0FDF00050FC6F580807E1FD5108
:105BB000020804E1FE5302E1FF5329E0D892196A7A
:105BC000F2BE198EF29E24C045F123C044F122C0DA
:105BD00043F121C042F10101496B486B476B0A0E4A
:105BE000466F0001E6EC11F019BEF28E03C0FFF023
:105BF00002C0FEF001C0FDF00050FC6FD0083CE197
:105C0000FD51070839E1FE5337E1FF5335E1D892E2
:105C1000196AF2BE198EF29E24C045F123C044F1E8
:105C200022C043F121C042F10101496B486B476B2F
:105C30000A0E466F0001E6EC11F019BEF28E01C0AB
:105C4000CDF0D892196AF2BE198EF29E24C045F1A9
:105C500023C044F122C043F121C042F10101496B4C
:105C6000486B476B0A0E466F0001E6EC11F019BE57
:105C7000F28E00C0CEF004D0020ECD6F580ECE6F63
:105C8000050ECF6F6C0ED06F9C0ED16F250ED26FAC
:105C9000830ED36FD4D2150EBF6F020EC16F010EEB
:105CA000C26F200EC36FC46F300EC56FD892196AD1
:105CB000F2BE198EF29E24C045F123C044F122C0E9
:105CC00043F121C042F10101496B486B476B0A0E59
:105CD000466F0001E6EC11F019BEF28E03C0FFF032
:105CE00002C0FEF001C0FDF00050FC6FDC080AE1CC
:105CF000FD5308E1FE5306E1FF5304E1CD6BDC0EDA
:105D0000CE6F04D0010ECD6FB80ECE6F060ECF6FE2
:105D1000020ED06F1A0ED16FF90ED26F3F0ED36FF5
:105D2000D46B0E0ED56F050ED66F89D21F0EBF6FC6
:105D3000030EC16F010EC26F300EC36F200EC46F11
:105D4000C56FC66FC76FC86FC96FCA6FD892196A1F
:105D5000F2BE198EF29E24C045F123C044F122C048
:105D600043F121C042F10101496B486B476B0A0EB8
:105D7000466F0001E6EC11F019BEF28E03C0FFF091
:105D800002C0FEF001C0FDF00050FC6FB80806E153
:105D9000FD2D04D0FE5302E1FF5329E0D892196A89
:105DA000F2BE198EF29E24C045F123C044F122C0F8
:105DB00043F121C042F10101496B486B476B0A0E68
:105DC000466F0001E6EC11F019BEF28E03C0FFF041
:105DD00002C0FEF001C0FDF00050FC6FD0083CE1B5
:105DE000FD51070839E1FE5337E1FF5335E1D89201
:105DF000196AF2BE198EF29E24C045F123C044F107
:105E000022C043F121C042F10101496B486B476B4D
:105E10000A0E466F0001E6EC11F019BEF28E01C0C9
:105E2000CDF0D892196AF2BE198EF29E24C045F1C7
:105E300023C044F122C043F121C042F10101496B6A
:105E4000486B476B0A0E466F0001E6EC11F019BE75
:105E5000F28E00C0CEF004D0010ECD6FB80ECE6F22
:105E6000050ECF6F630ED06F6E0ED16F310ED26FF5
:105E70003D0ED36FE4D1270EBF6F0A0EC06FC16B0A
:105E8000010EC26F310EC36F370EC46F320EC56F75
:105E9000330EC66F380EC76F320EC86F300EC96F23
:105EA000310ECA6FD892196AF2BE198EF29E24C0C2
:105EB00045F123C044F122C043F121C042F1010168
:105EC000496B486B476B0A0E466F0001E6EC11F018
:105ED00019BEF28E03C0FFF002C0FEF001C0FDF05B
:105EE0000050FC6FB80806E1FD2D04D0FE5302E11E
:105EF000FF5329E0D892196AF2BE198EF29E24C08F
:105F000045F123C044F122C043F121C042F1010117
:105F1000496B486B476B0A0E466F0001E6EC11F0C7
:105F200019BEF28E03C0FFF002C0FEF001C0FDF00A
:105F30000050FC6FD0083CE1FD51070839E1FE53E9
:105F400037E1FF5335E1D892196AF2BE198EF29EFD
:105F500024C045F123C044F122C043F121C042F1E5
:105F60000101496B486B476B0A0E466F0001E6EC76
:105F700011F019BEF28E01C0CDF0D892196AF2BEAE
:105F8000198EF29E24C045F123C044F122C043F192
:105F900021C042F10101496B486B476B0A0E466F05
:105FA0000001E6EC11F019BEF28E00C0CEF004D074
:105FB000010ECD6FB80ECE6F050ECF6F630ED06F92
:105FC0006E0ED16F310ED26F3D0ED36F38D1280EC9
:105FD000BF6F0A0EC16F010EC26F430EC36F330E47
:105FE000C46F300EC56FC66F2A0EC76F200EC86F04
:105FF000390EC96F310ECA6F020ECD6F580ECE6FBB
:10600000050ECF6FFA0ED06F830ED16F690ED26F6F
:10601000350ED36F14D1280EBF6F0A0EC16F010E5B
:10602000C26F430EC36F330EC46F300EC56FC66FA1
:106030002A0EC76F200EC86F390EC96F310ECA6F96
:10604000050ECF6FCD6BDC0ECE6FFA0ED06F830EC8
:10605000D16F690ED26F350ED36FF1D0260EBF6FA0
:106060000A0EC16F010EC26F430EC36F330EC46FB1
:10607000300EC56FC66F2A0EC76F200EC86F390E5F
:10608000C96F310ECA6F020ECD6F580ECE6F050E5E
:10609000CF6FFA0ED06F830ED16F690ED26F350EAF
:1060A000D36FCDD0260EBF6F0A0EC16F010EC26F27
:1060B000440EC36F300EC46F310EC56F300EC66F05
:1060C0002A0EC76F310EC86F300EC96F590ECA6FD6
:1060D000CD6BDC0ECE6F050ECF6FFD0ED06F840E34
:1060E000D16F560ED26F380ED36FA9D0090EBF6F85
:1060F000050EC16F010EC26F300EC36F380EC46F34
:10610000300EC56F350EC66F320EC76F300EC86FBA
:10611000200EC96FCA6FD892196AF2BE198EF29E0C
:1061200024C045F123C044F122C043F121C042F113
:106130000101496B486B476B0A0E466F0001E6ECA4
:1061400011F019BEF28E03C0FFF002C0FEF001C0D4
:10615000FDF00050FC6FDC0806E1FD5304E1FE5346
:1061600002E1FF5328E0D892196AF2BE198EF29E1E
:1061700024C045F123C044F122C043F121C042F1C3
:106180000101496B486B476B0A0E466F0001E6EC54
:1061900011F019BEF28E03C0FFF002C0FEF001C084
:1061A000FDF00050FC6FB8083BE1FD2D39D0FE53E7
:1061B00037E1FF5335E1D892196AF2BE198EF29E8B
:1061C00024C045F123C044F122C043F121C042F173
:1061D0000101496B486B476B0A0E466F0001E6EC04
:1061E00011F019BEF28E01C0CDF0D892196AF2BE3C
:1061F000198EF29E24C045F123C044F122C043F120
:1062000021C042F10101496B486B476B0A0E466F92
:106210000001E6EC11F019BEF28E00C0CEF004D001
:10622000010ECD6FB80ECE6F040ECF6FCF0ED06FB4
:106230006F0ED16FDF0ED26F410ED36F00D0BE5103
:10624000F00F32E2100FB7EF34F0010EC06F2CD018
:10625000020EC06F29D0030EC06F26D0040EC06F8F
:1062600023D0050EC06F20D0060EC06F1DD00F0EBC
:10627000C06F1C50030817E1870EC16F420EC26F3A
:10628000200EC36F330ECA6F050ECF6F6B0ED06F2B
:10629000080ED16FFA0ED26F380ED36FD46B050E85
:1062A000D56FF60ED66F00D0CDC0F3F0CEC0F2F0B1
:1062B0001AAE39D0F3C0FDF0F2C0FCF0FF6B0A0E4D
:1062C000FE6FE4EC20F002C0DBF0F3C0FDF0F2C0A2
:1062D000FCF0FF6B0A0EFE6FE4EC20F001C0DCF076
:1062E000196AF2BE198EF29EF3C038F1F2C037F18E
:1062F000010E01013A6FB80E396F000140EC1BF03E
:1063000019BEF28E02C003F001C0FCF002C0FDF025
:10631000F3EC20F003C0FBF002C0FAF001C0F9F08A
:1063200000C0F8F0ABD02150DD080DE12250260866
:106330000AE1235208E1245206E1D96B110EDB6F0A
:10634000300EDC6F9BD023C0D9F022C0DBF021C01F
:10635000DCF0D892196AF2BE198EF29E24C045F183
:1063600023C044F122C043F121C042F10101496B35
:10637000486B476B0A0E466F0001E6EC11F019BE40
:10638000F28E03C0FFF002C0FEF001C0FDF000C0BD
:10639000FCF0FF5309E1FE5307E1F351FD5D69E3B2
:1063A00003E1FC51F25D65E2D892196AF2BE198EE2
:1063B000F29E24C045F123C044F122C043F121C024
:1063C00042F10101496B486B476B0A0E466F0001B1
:1063D000E6EC11F019BEF28E03C0FFF002C0FEF031
:1063E00001C0FDF000C0FCF00EEF21F003C0FBF097
:1063F00002C0FAF001C0F9F000C0F8F0F3C0FDF0FF
:10640000F2C0FCF0F3EC20F0FBC0FFF0FAC0FEF0AD
:10641000F9C0FDF0F8C0FCF003C003F102C002F1C6
:1064200001C001F100C000F129EF21F000C0FCF033
:1064300001C0FDF002C0FEF003C0FFF0D89203C01F
:1064400003F102C002F101C001F100C000F101013D
:10645000076B066B056B7F0E046F0001E8EF21F000
:1064600003C0FBF002C0FAF001C0F9F000C0F8F080
:1064700005D0FB6BFA6BF96B7F0EF86FFD6BBF0EEF
:10648000FC6FBEC0FEF025EF23F018EC11F01ABE31
:10649000E7D1380EF66E1C0EF76E196AF2BE198E31
:1064A000F29EB4EC11F019BEF28E2EEC25F0196AB2
:1064B000F2BE198EF29E16EC1AF019BEF28E01523F
:1064C000F6E0196AF2BE198EF29E990E0101376F3D
:1064D000000180EC1AF019BEF28E0400200E006E4E
:1064E000002EFED700D0F06BF0512F08D8A0AAD014
:1064F00004003EEC25F0036AF051BF0FE96E000E78
:106500000320EA6EEFCFFCF0196AF2BE198EF29EFC
:10651000F0C03AF1370E01013B6F00011BEC1BF09C
:1065200019BEF28E3A0E04009EA8FDD7AD6E196A10
:10653000F2BE198EF29EFCC03AF1370E01013B6F9C
:1065400000011BEC1BF019BEF28E200E04009EA869
:10655000FDD7AD6E2D0E04009EA8FDD7AD6E200EAA
:1065600004009EA8FDD7AD6E036AF051BF0FE96E1F
:10657000000E0320EA6EEFCFFCF0196AF2BE198E0E
:10658000F29EFCC037F180EC1AF019BEF28E0400C6
:10659000100E006E002EFED7196AF2BE198EF29E02
:1065A000F9EC1AF019BEF28E01C0F1F0036AF05155
:1065B000BF0FE96E000E0320EA6EEF50F15D39E186
:1065C000196AF2BE198EF29E770E0101376F000133
:1065D00080EC1AF019BEF28E196AF2BE198EF29E84
:1065E000F1C03AF1370E01013B6F00011BEC1BF0CB
:1065F00019BEF28E0D0E04009EA8FDD7AD6E0A0ED8
:1066000004009EA8FDD7AD6E196AF2BE198EF29EE7
:10661000040E0101396F0001FEEC19F019BEF28E73
:10662000196AF2BE198EF29EF9EC1AF019BEF28EBA
:1066300007D00400200E006E002EFED700D058D7E1
:10664000F02B52D72150DD080FE1225026080CE133
:1066500023520AE1245208E11E0EFC6FFD6B010E6D
:10666000FE6F4EEC25F0FBD0FBC0FFF0FAC0FEF051
:10667000F9C0FDF0F8C0FCF058EC26F001C0EFF0D6
:10668000F2CFFCF0F29EAA6A040EA96EA69CA69E0A
:10669000A680A850FCBFF28EFD6FF2CFFEF0F29EF6
:1066A000AA6A030EA96EA69CA69EA680A850FEBF4D
:1066B000F28EFF6FF2CF00F1F29EAA6A020EA96E6F
:1066C000A69CA69EA680A850010100BFF28E016F75
:1066D000F2CF02F1F29EAA6A010EA96EA69CA69EB6
:1066E000A680A85002BFF28E036FFDC0F7F0FFC076
:1066F000F6F001C1F5F003C1F4F00001EF51F42709
:10670000000EF523F623F723F7C0FDF0FE6BFF6BB9
:106710000101006BAA6A040EA96EFDC0A8FFA69C29
:10672000A69EA684F250006EF29E0F01550EA76E33
:10673000AA0EA76EA682A6B2FED7A6940050F212A9
:10674000F6C0FDF0F7C0FEF00001FF6B0101006B29
:10675000AA6A030EA96EFDC0A8FFA69CA69EA684E9
:10676000F250006EF29E0F01550EA76EAA0EA76E94
:10677000A682A6B2FED7A6940050F212F5C0FDF094
:10678000F6C0FEF0F7C0FFF00101006BAA6A020E2E
:10679000A96EFDC0A8FFA69CA69EA684F250006E1E
:1067A000F29E0F01550EA76EAA0EA76EA682A6B284
:1067B000FED7A6940050F212AA6A010EA96EF4C088
:1067C000A8FFA69CA69EA684F2CF00F0F29E550ECE
:1067D000A76EAA0EA76EA682A6B2FED7A6940050F8
:1067E000F2120D0E04009EA8FDD7AD6E0A0E040035
:1067F0009EA8FDD7AD6EF2CFFCF0F29EAA6A160EEF
:10680000A96EA69CA69EA680A8500001FCBFF28E91
:10681000FD6FF2CFFEF0F29EAA6A170EA96EA69C3B
:10682000A69EA680A850FEBFF28EFF6FFDC003F0AB
:10683000FF51016EF351035C0CE303E10150F25D83
:1068400008E2EFC0FCF0FD6B010EFE6F4EEC25F090
:1068500006D0FC6BFD6B010EFE6F4EEC25F05BD09D
:10686000F06BF0511F0819E3036AF051250F016E18
:10687000000E032203C0FDF0036AF051BF0FE96E62
:10688000000E0320EA6EEFCFFEF0FDC0EAFF01C06C
:10689000E9FFFEC0EFFFF02BE4D7F06BF0511F08CB
:1068A00016E3FC6BF0C0FDF0080EFE6FFDEC27F068
:1068B000196AF2BE198EF29E010E0101396F0001B4
:1068C000FEEC19F019BEF28E080EF027E7D7FC6B2C
:1068D000FDEC28F0FAEC29F0196AF2BE198EF29E4E
:1068E0000101326B0001FDEC1BF019BEF28EFBC002
:1068F000FFF0FAC0FEF0F9C0FDF0F8C0FCF058EC73
:1069000026F001C0EFF0EFC0FCF0FD6B010EFE6F52
:106910004EEC25F01B921B92040EFC6F196AF2BE1E
:10692000198EF29EFA0E0101396F0001FEEC19F08A
:1069300019BEF28EFC2FF2D7000CE824F76AF73666
:10694000550FF66E690EF7220A00F550FA6E080030
:10695000F550F96EB25504575058F059425B2C5D12
:10696000765E965C1660CE5F5C60A460EC60E824A6
:10697000F76AF736890FF66E690EF7220A00F550AE
:10698000FA6E0800F550F96E5C624A625062566217
:1069900062626862A862A862A862A862A862A8622D
:1069A000A862A862A8626E62880EF66E120EF76E7A
:1069B000196AF2BE198EF29EB4EC11F019BEF28E75
:1069C00004009EAAFDD7AE50000C93908A9093804D
:1069D0000400200E006E002EFED700D09380C691DA
:1069E00081B0C68104003B0E006E002EFED7000071
:1069F000000EC6B1010E016E000C93908A90040047
:106A000000D000D0C75309E093908A800400200E84
:106A1000006E002EFED700D008D093908A9004001C
:106A2000200E006E002EFED700D00400330E006E44
:106A3000002EFED793800400090E006E002EFED7B4
:106A40000000000CC26B010EC36FC46B196AF2BE6A
:106A5000198EF29E16EC1AF019BEF28E015203E165
:106A6000000E016E31D1196AF2BE198EF29EF00E3F
:106A70000101376F000180EC1AF019BEF28E04009C
:106A8000100E006E002EFED7C3514008D8A013D1BF
:106A90009CDFC59101B0C58198DFC59301B0C58366
:106AA000C5A106D0C5A304D0C485C4C001F00CD1D3
:106AB000C5B196D0C5B394D0A651C35D22E1010EF5
:106AC000C35D006E0032003200321F0E001600500F
:106AD000036A450F016E000E032201C0E9FF03C0E7
:106AE000EAFF010EC35D070BC66F010E006EC651B3
:106AF000016E04E0D8900036012EFCD70050EF1252
:106B00004AD0C351A65D25E2010EC35D006E00327E
:106B1000003200321F0E00160050036A450F016E4E
:106B2000000E032201C0E9FF03C0EAFF010EC35DAE
:106B3000070BC66F010E006EC651016E04E0D890BF
:106B40000036012EFCD70050FF0AEF16C3C0C2F07A
:106B500022D0010EC35D006E0032003200321F0EE3
:106B600000160050036A450FE96E000E0320EA6E1E
:106B7000EFCFC6F0010EC35D070BC76FC6C000F0B4
:106B8000C751016E04E0D8900032012EFCD700B04E
:106B900002D0C3C0C2F0010EC35D006E00320032ED
:106BA00000321F0E00160050036A450FE96E000EFA
:106BB0000320EA6EEFCFC6F0010EC35D070BC76F6F
:106BC000C6C000F0C751016E04E0D8900032012E1B
:106BD000FCD7000E00B0010EC76F0FDFC32B6AD0C9
:106BE000C5A122D0010EC35D006E0032003200321A
:106BF0001F0E00160050036A450F016E000E03229F
:106C000001C0E9FF03C0EAFF010EC35D070BC66FB9
:106C1000010E006EC651016E04E0D8900036012EC0
:106C2000FCD70050EF1222D0010EC35D006E00327F
:106C3000003200321F0E00160050036A450F016E2D
:106C4000000E032201C0E9FF03C0EAFF010EC35D8D
:106C5000070BC66F010E006EC651016E04E0D8909E
:106C60000036012EFCD70050FF0AEF16010EC35D5F
:106C7000006E0032003200321F0E00160050036A10
:106C8000450FE96E000E0320EA6EEFCFC6F0010E4D
:106C9000C35D070BC76FC6C000F0C751016E04E0AB
:106CA000D8900032012EFCD7000E00B0010EC76F45
:106CB000A4DEC32BE9D6C2C0A6F0A65302E1C4816C
:106CC00001D0C483C4C001F092EF36F0BF6BBF5156
:106CD00009081AE3C06BC051070814E3BF51080D3F
:106CE000F350C36BC26F036AC051C225016EC3511A
:106CF00003220150550FE96E000E0320EA6EEF6A81
:106D0000C02BE9D7BF2BE3D7010EBF6F0D0E0400D8
:106D10009EA8FDD7AD6E0A0E04009EA8FDD7AD6EED
:106D2000A66B90D60150FB0FD8B0CCD0050F9CEFCE
:106D300037F0F40EF66E100EF76E196AF2BE198E69
:106D4000F29EB4EC11F019BEF28EF4D0BE531EE0E8
:106D5000196AF2BE198EF29EBFC038F1110E010100
:106D6000396F000143EC11F019BEF28E170EF66E6A
:106D7000110EF76E196AF2BE198EF29E040E010111
:106D8000396F0001EAEC13F019BEF28EC06BC051EE
:106D9000070824E3010EBF5D080DF350C36BC26FFB
:106DA000036AC051C225016EC35103220150550F21
:106DB000016E000E032203C0C3F0036AC051450FE9
:106DC000E96E000E0320EA6EEFCFC4F0C3C0EAFF05
:106DD00001C0E9FFC4C0EFFFC02BD9D7BE530BE001
:106DE000196AF2BE198EF29E0101376B000163EC45
:106DF0001BF019BEF28EC19165D0BE531EE0196A18
:106E0000F2BE198EF29EBFC038F1110E0101396F2A
:106E1000000143EC11F019BEF28E1F0EF66E110E3A
:106E2000F76E196AF2BE198EF29E040E0101396FD7
:106E30000001EAEC13F019BEF28EC06BC0510708D6
:106E400024E3010EBF5D080DF350C36BC26F036AEC
:106E5000C051C225016EC35103220150550F016E6E
:106E6000000E032203C0C3F0036AC051450FE96E50
:106E7000000E0320EA6EEFCFC4F0C3C0EAFF01C0EA
:106E8000E9FFC4C0EFFFC02BD9D7BE530BE0196A8E
:106E9000F2BE198EF29E0101376B000163EC1BF00C
:106EA00019BEF28EBF2BC1810DD0240EF66E110ECD
:106EB000F76E196AF2BE198EF29EB4EC11F019BE8B
:106EC000F28E38D0C1A101D02CD7BE5332E0580E7B
:106ED000F66E110EF76E196AF2BE198EF29EB4ECC0
:106EE00011F019BEF28EA60EF66E110EF76E196A2B
:106EF000F2BE198EF29EB4EC11F019BEF28EEE0EB7
:106F0000F66E110EF76E196AF2BE198EF29EB4EC8F
:106F100011F019BEF28EE8EC27F001C0C0F0C051AC
:106F2000BF5D03E2FF0EA56F03D0010EBF5DA56F2D
:106F300001D0A56B45EF53F0E824F76AF736530FFD
:106F4000F66E6F0EF7220A00F550FA6E0800F55043
:106F5000F96E326D4C6DFA6DC46EAA6EE851EA1985
:106F6000800BEC6FE8AF05D0E71FE81FE72BD8B424
:106F7000E82BEAAF05D0E91FEA1FE92BD8B4EA2BCA
:106F8000E751E903F3CF01F0F4CF00F0EA03F35047
:106F90000026E851E903F3500020026EECAF05D063
:106FA000011E021E012AD8B4022A48EF38F0E56B10
:106FB000E36B0A0EE46FE26BE16BDF51E01104E179
:106FC000000E016E026EE6D0E551E52B036ADF2567
:106FD000E96EE0510320EA6EEFCFE6F0E6512D08AE
:106FE0000DE1010EE36FE551E52B036ADF25E96E44
:106FF000E0510320EA6EEFCFE6F00DD0E6512B080A
:107000000AE1E551E52B036ADF25E96EE051032033
:10701000EA6EEFCFE6F0E6512F08D8B0ADD0E651DA
:107020003908D8A0A9D0E651300821E1036AE5511A
:10703000DF25E96EE0510320EA6EEF5078080AE0A0
:10704000036AE551DF25E96EE0510320EA6EEF5057
:1070500058080DE1100EE46FE52BE551E52B036AAE
:10706000DF25E96EE0510320EA6EEFCFE6F0E45150
:107070000A0821E1E6512F081DE2E65139081AE31A
:10708000E86B0A0EE76FE2C0EAF0E1C0E9F066D70C
:10709000300EE65D0124E16F000E0220E26FE55143
:1070A000E52B036ADF25E96EE0510320EA6EEFCF9E
:1070B000E6F0E0D761D0E45110085EE1E6516008E7
:1070C00006E2E6517A0803E3E651DF0B01D0E65110
:1070D000E66FE6512F0803E2E651390806E2E65171
:1070E00040084AE2E651460847E3E6512F0819E214
:1070F000E651390816E3E135E76FE235E86FE73727
:10710000E837E737E837E737E837F00EE717300EAC
:10711000E65DE725016E000EE82101C0E1F0E26FB7
:1071200016D0E135E76FE235E86FE737E837E73744
:10713000E837E737E837F00EE717410EE65D0A0F4C
:10714000E725016E000EE82101C0E1F0E26FE55194
:10715000E52B036ADF25E96EE0510320EA6EEF506C
:10716000E66F600806E2E6517A0803E3E651DF0BBA
:1071700001D0E651E66FADD7E4510A0807E1E32DEF
:1071800005D0E11FE21FE12BD8B4E22BE1C001F0F2
:10719000E2C002F0D9EF38F00101086BD60E076F9C
:1071A000070E096F0001B1EC26F0E06BD60EDF6F21
:1071B000FED602C0DEF001C0DDF0DDC001F0DEC0B1
:1071C00002F0000C010E0101296F2951285D07E32F
:1071D00024312733263325332433292BF6D724C1F2
:1071E00000F025C101F026C102F027C103F0000123
:1071F000000C010E0101296F2951285D07E3273595
:107200002437253726372737292BF6D724C100F016
:1072100025C101F026C102F027C103F00001000CD6
:10722000120EE16F340EE06F560EDF6F780EDE6FD8
:10723000010EDC6FDC510A083AE3DC51040DF35017
:10724000036ADE0F016E000E032201C01EF103C0AF
:107250001FF1010E0001DC5D040DF350036ADE0F27
:10726000E96E000E0320EA6EEFCF20F1ECCF21F1A2
:10727000ECCF22F1ECCF23F123C127F122C126F17B
:1072800021C125F120C124F1020E0101286F000166
:1072900099DF1FC1EAFF1EC1E9FF00C0EFFF01C077
:1072A000ECFF02C0ECFF03C0ECFFDC2BC3D7F2CF36
:1072B0001EF1F29EAA6A200EA96EA69CA69EA6802A
:1072C000A85001011EBFF28E1F6FF2CF20F1F29E77
:1072D000AA6A210EA96EA69CA69EA680A85020BFD1
:1072E000F28E216FD6C00CF1D7C00DF11FC10BF18A
:1072F00021C10AF19A0E116FBC0E106FDE0E0F6FD6
:10730000F00E0E6FF2CF1EF1F29EAA6A220EA96E47
:10731000A69CA69EA680A8501EBFF28E1F6F1FC1FE
:1073200015F1FF0E146FFF0E136F800E126F196BA5
:10733000186B176B166B1D6B1C6B010E1B6FB80E59
:107340001A6F670E0001AA6F450EA96F230EA86F72
:10735000010EA76FEF0EAE6FCD0EAD6FAB0EAC6F23
:10736000890EAB6F980EB26FBA0EB16FDC0EB06FB4
:10737000FE0EAF6F100EB66F320EB56F540EB46FB7
:10738000760EB36FC30EBA6FD20EB96FE10EB86F3F
:10739000F00EB76FDC6BDC514F08D8A04CD3DC513A
:1073A0000F0BDD6FDC510F08D8B08CD0DD51040D10
:1073B000F350036ADE0F016E000E032201C01EF1BE
:1073C00003C01FF10D0E0001DD250F0B040DF3505E
:1073D000036ADE0FE96E000E0320EA6EEFCF20F1A4
:1073E000ECCF21F1ECCF22F1ECCF23F1080EDD251B
:1073F0000F0B040DF350036ADE0FE96E000E03203D
:10740000EA6EEFCF00F0ECCF01F0ECCF02F0ECCF62
:1074100003F000500101201B0150211B0250221BD0
:107420000350231B020E0001DD250F0B040DF3504A
:10743000036ADE0FE96E000E0320EA6EEFCF00F064
:10744000ECCF01F0ECCF02F0ECCF03F000500101E3
:10745000201B0150211B0250221B0350231B000143
:10746000DD51040DF350036ADE0FE96E000E0320B8
:10747000EA6EEFCF00F0ECCF01F0ECCF02F0ECCFF2
:1074800003F000500101201B0150211B0250221B60
:107490000350231B23C127F122C126F121C125F16D
:1074A00020C124F1010E286F0001A3DE1FC1EAFFF5
:1074B0001EC1E9FF00C0EFFF01C0ECFF02C0ECFFFE
:1074C00003C0ECFFDC51130802E2000E01D0010EF4
:1074D000010BD8B49ED0AAC027F1A9C026F1A8C03C
:1074E00025F1A7C024F1050E0101286F000181DEFE
:1074F00003C021F102C020F101C01FF100C01EF144
:10750000AB51AF150101226F0001AC51B015010163
:10751000236F0001AD51B1150101246F0001AE517F
:10752000B2150101256FABC026F10101261FACC0C9
:1075300027F10101271FADC028F10101281FAEC0AE
:1075400029F10101291F26510001B315006E010127
:1075500027510001B415016E010128510001B51534
:10756000026E010129510001B615036E00500101A0
:107570002211006E01502311016E02502411026E7F
:1075800003502511036E00501E2701501F23025087
:107590002023035021230001B75101011E270001C0
:1075A000B85101011F230001B9510101202300013D
:1075B000BA51010121230001DD51040DF350036A8A
:1075C000DE0FE96E000E0320EA6EEFCF00F0ECCF85
:1075D00001F0ECCF02F0ECCF03F0005001011E27C8
:1075E00001501F230250202303502123990E1E25F2
:1075F0000001D86F790E01011F210001D96F820EA1
:10760000010120210001DA6F5A0E01012121000140
:10761000DB6FDC51130802E3000E01D0010E010103
:107620001E6F0001DC51270802E2000E01D0010E9E
:1076300001011E15D8B481D0AAC027F1A9C026F136
:10764000A8C025F1A7C024F1050E286F0001D1DDE7
:1076500003C021F102C020F101C01FF100C01EF1E2
:10766000AB51AF190101226F0001AC51B0190101FA
:10767000236F0001AD51B1190101246F0001AE511A
:10768000B2190101256F22510001B319006E0101E9
:1076900023510001B419016E010124510001B519F3
:1076A000026E010125510001B619036E005001015F
:1076B0001E2701501F2302502023035021230001C5
:1076C000B75101011E270001B85101011F2300011C
:1076D000B951010120230001BA5101012123000108
:1076E000DD51040DF350036ADE0FE96E000E032036
:1076F000EA6EEFCF00F0ECCF01F0ECCF02F0ECCF70
:1077000003F0005001011E2701501F2302502023C7
:1077100003502123A10E1E250001D86FEB0E01019D
:107720001F210001D96FD90E010120210001DA6F5C
:107730006E0E010121210001DB6F0001DC512708E1
:1077400002E3000E01D0010E01011E6F0001DC51A9
:107750003B0802E2000E01D0010E01011E15D8B453
:107760009DD0AAC027F1A9C026F1A8C025F1A7C0C5
:1077700024F1050E286F00013CDD03C021F102C099
:1077800020F101C01FF100C01EF1AB51AF15010186
:10779000226F0001AC51B0150101236F0001AD5102
:1077A000B1150101246F0001AE51B2150101256F21
:1077B0000001AB51B315006EAC51B415016EAD5163
:1077C000B515026EAE51B615036E005001012213BD
:1077D0000150231302502413035025130001AF510D
:1077E000B315006EB051B415016EB151B515026EEE
:1077F000B251B615036E005001012211006E015006
:107800002311016E02502411026E03502511036EE4
:1078100000501E2701501F23025020230350212314
:107820000001B75101011E270001B85101011F23BA
:107830000001B951010120230001BA5101012123A6
:107840000001DD51040DF350036ADE0FE96E000EF6
:107850000320EA6EEFCF00F0ECCF01F0ECCF02F0A6
:10786000ECCF03F0005001011E2701501F230250EE
:10787000202303502123DC0E1E250001D86FBC0EEF
:1078800001011F210001D96F1B0E01012021000100
:10789000DA6F8F0E010121210001DB6F0001DC5145
:1078A0003B0802E3000E01D0010E01011E6F000132
:1078B000DC514F0802E2000E01D0010E01011E153D
:1078C000D8B482D0AAC027F1A9C026F1A8C025F15A
:1078D000A7C024F1050E286F00018BDC03C021F145
:1078E00002C020F101C01FF100C01EF1AB51AF1961
:1078F0000101226F0001AC51B0190101236F000199
:10790000AD51B1190101246F0001AE51B21901014D
:10791000256F22510001B319006E010123510001AE
:10792000B419016E010124510001B519026E010163
:1079300025510001B619036E005001011E270150A8
:107940001F2302502023035021230001B7510101BE
:107950001E270001B85101011F230001B951010187
:1079600020230001BA51010121230001DD51040D42
:10797000F350036ADE0FE96E000E0320EA6EEFCFCC
:1079800000F0ECCF01F0ECCF02F0ECCF03F00050B0
:1079900001011E2701501F230250202303502123E1
:1079A000D60E1E250001D86FC10E01011F21000156
:1079B000D96F620E010120210001DA6FCA0E0101A8
:1079C00021210001DB6F0101B6C0BAF0B5C0B9F0EA
:1079D000B4C0B8F0B3C0B7F0B2C0B6F0B1C0B5F043
:1079E000B0C0B4F0AFC0B3F0AEC027F1ADC026F167
:1079F000ACC025F1ABC024F1020E286F0001E2EC0F
:107A000038F003C0B2F002C0B1F001C0B0F000C065
:107A1000AFF0AAC0AEF0A9C0ADF0A8C0ACF0A7C04E
:107A2000ABF0DBC0AAF0DAC0A9F0D9C0A8F0D8C08A
:107A3000A7F0DC2BB0D415EF3EF018EC11F0F2CF2C
:107A4000D6F0F29EAA6A200EA96EA69CA69EA680DB
:107A5000A850D6BFF28ED76FF2CFD8F0F29EAA6AA6
:107A6000210EA96EA69CA69EA680A850D8BFF28E15
:107A7000D96FD7C0DBF0D9C0DAF0F2CFDCF0F29EDC
:107A8000AA6A220EA96EA69CA69EA680A850DCBF5C
:107A9000F28EDD6F700EF66E150EF76E196AF2BE7D
:107AA000198EF29E150E0101396F0001EAEC13F0F8
:107AB00019BEF28E100EE96E196AF2BE198EF29E90
:107AC000DBC03BF1DAC03AF18FEC12F019BEF28E56
:107AD000880EF66E150EF76E196AF2BE198EF29EBA
:107AE0000D0E0101396F0001EAEC13F019BEF28EA0
:107AF000196AF2BE198EF29EDDC038F11B0E01012B
:107B0000396F000143EC11F019BEF28E0D0E040026
:107B10009EA8FDD7AD6E0A0E04009EA8FDD7AD6EDF
:107B20000A0E04009EA8FDD7AD6E9C0EF66E150ED3
:107B3000F76E196AF2BE198EF29EB4EC11F019BEFE
:107B4000F28EEA0EF66E150EF76E196AF2BE198EF7
:107B5000F29EB4EC11F019BEF28EF2CFD6F0F29E86
:107B6000AA6A100EA96EA69CA69EA680A850D6BF93
:107B7000F28ED76FF2CFD8F0F29EAA6A110EA96EDC
:107B8000A69CA69EA680A850D8BFF28ED96FD7C05B
:107B9000C1F0D9C0C0F0380EF66E160EF76E196A35
:107BA000F2BE198EF29E130E0101396F0001EAEC4C
:107BB00013F019BEF28E100EE96E196AF2BE198E1C
:107BC000F29EC1C03BF1C0C03AF18FEC12F019BE79
:107BD000F28E0D0E04009EA8FDD7AD6E0A0E0400B5
:107BE0009EA8FDD7AD6E0A0E04009EA8FDD7AD6E0F
:107BF000520EF66E160EF76E196AF2BE198EF29ECE
:107C0000B4EC11F019BEF28ECCEC38F002C0BFF02B
:107C100001C0BEF0BE5303E1BF5301E19DD1BFC01F
:107C2000D7F0BEC0D6F010EF39F08A0EF66E160E01
:107C3000F76E196AF2BE198EF29EB4EC11F019BEFD
:107C4000F28EE20EF66E0F0EF76E196AF2BE198E04
:107C5000F29EB4EC11F019BEF28EB80EF66E160E4E
:107C6000F76E196AF2BE198EF29EB4EC11F019BECD
:107C7000F28E9BEC26F001C0D6F09BEC26F001C002
:107C8000D7F09BEC26F001C0D8F09BEC26F0D6C0D4
:107C9000C5F0D7C0C4F0D8C0C3F001C0C2F09BEC9F
:107CA00026F001C0D6F09BEC26F001C0D7F09BEC8B
:107CB00026F001C0D8F09BEC26F0D6C0C9F0D7C0A2
:107CC000C8F0D8C0C7F001C0C6F09BEC26F001C0D8
:107CD000D6F09BEC26F001C0D7F09BEC26F001C05B
:107CE000D8F09BEC26F0D6C0CDF0D7C0CCF0D8C0F1
:107CF000CBF001C0CAF09BEC26F001C0D6F09BECA3
:107D000026F001C0D7F09BEC26F001C0D8F09BEC28
:107D100026F0D6C0D1F0D7C0D0F0D8C0CFF001C087
:107D2000CEF09BEC26F001C0D6F09BEC26F001C013
:107D3000D7F09BEC26F001C0D8F09BEC26F0D6C023
:107D4000D5F0D7C0D4F0D8C0D3F001C0D2F0A7513D
:107D5000C25DD8A4E5D0A851C35DD8A4E1D0A95193
:107D6000C45DD8A4DDD0AA51C55DD8A4D9D0AB518B
:107D7000C65DD8A4D5D0AC51C75DD8A4D1D0AD5183
:107D8000C85DD8A4CDD0AE51C95DD8A4C9D0AF517B
:107D9000CA5DD8A4C5D0B051CB5DD8A4C1D0B15173
:107DA000CC5DD8A4BDD0B251CD5DD8A4B9D0B3516B
:107DB000CE5DD8A4B5D0B451CF5DD8A4B1D0B55163
:107DC000D05DD8A4ADD0B651D15DD8A4A9D0B7515B
:107DD000D25DD8A4A5D0B851D35DD8A4A1D0B95153
:107DE000D45DD8A49DD0BA51D55DD8A499D0C05146
:107DF000BE27C151BF23BFC0D6F0D76BAA6A100EF1
:107E0000A96ED6C0A8FFA69CA69EA684F250006EBE
:107E1000F29E0F01550EA76EAA0EA76EA682A6B2FD
:107E2000FED7A6940050F212AA6A110EA96EBEC027
:107E3000A8FFA69CA69EA684F2CF00F0F29E550E47
:107E4000A76EAA0EA76EA682A6B2FED7A694005071
:107E5000F212F2CFD6F0F29EAA6A220EA96EA69C6A
:107E6000A69EA680A8500001D6BFF28E010FD76F44
:107E7000AA6A220EA96ED7C0A8FFA69CA69EA684B9
:107E8000F250006EF29E0F01550EA76EAA0EA76E5D
:107E9000A682A6B2FED7A6940050F212BE0EF66ECF
:107EA000160EF76E196AF2BE198EF29E2B0E0101A4
:107EB000396F0001EAEC13F019BEF28E100EE96E74
:107EC000196AF2BE198EF29EC1C03BF1C0C03AF1F0
:107ED0008FEC12F019BEF28EEC0EF66E160EF76EE7
:107EE000196AF2BE198EF29E040E0101396F00016B
:107EF000EAEC13F019BEF28E100EE96E196AF2BEAA
:107F0000198EF29EBFC03BF1BEC03AF18FEC12F069
:107F100019BEF28E2E0E04009EA8FDD7AD6E0CD0B9
:107F2000F60EF66E160EF76E196AF2BE198EF29EF6
:107F3000B4EC11F019BEF28E080ED66F196AF2BEBB
:107F4000198EF29EFA0E0101396F0001FEEC19F054
:107F500019BEF28ED62FF2D715EF54F0BE530CE0B7
:107F60009C0EF66E190EF76E196AF2BE198EF29E0D
:107F7000B4EC11F019BEF28EA53D01D009D0196AFA
:107F8000F2BE198EF29EB9EC1AF019BEF28E23D011
:107F9000196AF2BE198EF29E16EC1AF019BEF28E14
:107FA0000152F6E00400196AF2BE198EF29EDD0E4F
:107FB0000101396F0001D1EC10F019BEF28E196A7F
:107FC000F2BE198EF29ECC0E0101376F000180ECDB
:107FD0001AF019BEF28E0400090E006E002EFED7B4
:107FE0000000196AF2BE198EF29EC30E0101376FAE
:107FF000000180EC1AF019BEF28E0400090E006E2A
:10800000002EFED70000196AF2BE198EF29E010101
:10801000376B000180EC1AF019BEF28EBE530CE0F3
:10802000BA0EF66E190EF76E196AF2BE198EF29E2E
:10803000B4EC11F019BEF28EBF6BBF51070840E3DC
:108040000400090E006E002EFED70000280EBF258A
:10805000036A250F016E000E032201C0C0F003C0A9
:10806000C1F0196AF2BE198EF29EF9EC1AF019BE2F
:10807000F28EC1C0EAFFC0C0E9FF01C0EFFFBE53EE
:108080001DE0280EBF25036A250FE96E000E0320B0
:10809000EA6EEFCFC0F0196AF2BE198EF29EC0C030
:1080A0003AF1370E01013B6F00011BEC1BF019BECA
:1080B000F28E200E04009EA8FDD7AD6EBF2BBDD75B
:1080C000BE530FE00D0E04009EA8FDD7AD6E0A0E44
:1080D00004009EA8FDD7AD6E0A0E04009EA8FDD731
:1080E000AD6E41EF54F0A53D01D009D0196AF2BE42
:1080F000198EF29EB9EC1AF019BEF28E23D0196ACD
:10810000F2BE198EF29E16EC1AF019BEF28E0152D2
:10811000F6E00400196AF2BE198EF29EDD0E01012E
:10812000396F0001D1EC10F019BEF28E196AF2BE5F
:10813000198EF29ECC0E0101376F000180EC1AF00F
:1081400019BEF28E0400090E006E002EFED700004C
:10815000196AF2BE198EF29E5A0E0101376F0001A4
:1081600080EC1AF019BEF28E0400090E006E002E8B
:10817000FED70000196AF2BE198EF29EA50E01010B
:10818000376F000180EC1AF019BEF28E0400090E60
:10819000006E002EFED70000C20EF66E190EF76EAE
:1081A000196AF2BE198EF29EB4EC11F019BEF28E6D
:1081B000000CBE53D8A4ECD018EC11F0196AF2BE32
:1081C000198EF29E010E0101356F250E366F280EB5
:1081D000376F000185EC11F019BEF28EF20EF66ECB
:1081E000190EF76E196AF2BE198EF29EB4EC11F0F8
:1081F00019BEF28E196AF2BE198EF29EC6EC11F00B
:1082000019BEF28E1C0EF66E1A0EF76E196AF2BEC9
:10821000198EF29EB4EC11F019BEF28E460EF66E77
:108220001A0EF76E196AF2BE198EF29EB4EC11F0B6
:1082300019BEF28E196AF2BE198EF29E010E01016C
:10824000356F250E366F280E376F000185EC11F063
:1082500019BEF28E9BEC26F001C0BFF0196AF2BE87
:10826000198EF29EC6EC11F019BEF28EBF510708AE
:1082700001E2D4D7280EBF27660EF66E1A0EF76EEF
:10828000196AF2BE198EF29EB4EC11F019BEF28E8C
:10829000196AF2BE198EF29E010E0101356F250E8C
:1082A000366F280E376F000185EC11F019BEF28E83
:1082B000E8EC27F001C0C0F0196AF2BE198EF29EF8
:1082C000C6EC11F019BEF28EBF51C027BFC0C1F07D
:1082D000C051C15D5CE2C1511F0BC26F840EF66ECE
:1082E0001A0EF76E196AF2BE198EF29E1E0E010169
:1082F000396F0001EAEC13F019BEF28E196AF2BE72
:10830000198EF29EC2C03AF1370E01013B6F000197
:108310001BEC1BF019BEF28E3A0E04009EA8FDD78E
:10832000AD6E2D0E04009EA8FDD7AD6E200E04008C
:108330009EA8FDD7AD6E196AF2BE198EF29E010E8F
:108340000101356F250E366F280E376F000185EC61
:1083500011F019BEF28E036AC151250F016E000E95
:10836000032201C0C2F003C0C3F09BEC26F0C3C0DF
:10837000EAFFC2C0E9FF01C0EFFF196AF2BE198E21
:10838000F29EC6EC11F019BEF28EC12BA1D704D01B
:10839000280EBF6F2F0EC06FA53D01D009D0196AFE
:1083A000F2BE198EF29EB9EC1AF019BEF28E23D0ED
:1083B000196AF2BE198EF29E16EC1AF019BEF28EF0
:1083C0000152F6E00400196AF2BE198EF29EDD0E2B
:1083D0000101396F0001D1EC10F019BEF28E196A5B
:1083E000F2BE198EF29ECC0E0101376F000180ECB7
:1083F0001AF019BEF28E0400090E006E002EFED790
:108400000000196AF2BE198EF29E990E0101376FB3
:10841000000180EC1AF019BEF28E0400090E006E05
:10842000002EFED70000280EBF5DC26F196AF2BE93
:10843000198EF29EE8CF37F180EC1AF019BEF28E59
:10844000280EBF5DC26F196AF2BE198EF29EE8CF88
:108450003AF1370E01013B6F00011BEC1BF019BE16
:10846000F28E200E04009EA8FDD7AD6EBFC0C1F0F5
:10847000010EC025C15D37E20400090E006E002E1A
:10848000FED70000036AC151250FE96E000E0320DC
:10849000EA6EEFCFC2F0196AF2BE198EF29EC2C028
:1084A00037F180EC1AF019BEF28E036AC151250F24
:1084B000E96E000E0320EA6EEFCFC2F0196AF2BE39
:1084C000198EF29EC2C03AF1370E01013B6F0001D6
:1084D0001BEC1BF019BEF28E200E04009EA8FDD7E7
:1084E000AD6EC12BC5D7FFDD0D0E04009EA8FDD7D4
:1084F000AD6E0A0E04009EA8FDD7AD6E0A0E0400F4
:108500009EA8FDD7AD6E5CEF54F0A53D01D009D01B
:10851000196AF2BE198EF29EB9EC1AF019BEF28EEB
:1085200023D0196AF2BE198EF29E16EC1AF019BE0B
:10853000F28E0152F6E00400196AF2BE198EF29E24
:10854000DD0E0101396F0001D1EC10F019BEF28E81
:10855000196AF2BE198EF29ECC0E0101376F00012E
:1085600080EC1AF019BEF28E0400090E006E002E87
:10857000FED70000196AF2BE198EF29E660E010146
:10858000376F000180EC1AF019BEF28E0400090E5C
:10859000006E002EFED70000196AF2BE198EF29E00
:1085A0000101376B000180EC1AF019BEF28E040055
:1085B000090E006E002EFED70000196AF2BE198E59
:1085C000F29EF9EC1AF019BEF28E01C0BFF0BE5354
:1085D0004FE0360EF66E190EF76E196AF2BE198E5E
:1085E000F29E120E0101396F0001EAEC13F019BE80
:1085F000F28E196AF2BE198EF29EBFC03AF1370EA2
:1086000001013B6F00011BEC1BF019BEF28E200E26
:1086100004009EA8FDD7AD6EBF51030B0DE14E0EB9
:10862000F66E190EF76E196AF2BE198EF29EB4EC50
:1086300011F019BEF28E0CD0720EF66E190EF76E96
:10864000196AF2BE198EF29EB4EC11F019BEF28EC8
:108650000D0E04009EA8FDD7AD6E0A0E04009EA864
:10866000FDD7AD6E0A0E04009EA8FDD7AD6E09D0F1
:10867000BF3D04D0010E016E04D003D0000E016E88
:1086800000D087EF54F0BF6B010EBE6FBE510F08D4
:1086900056E393908A900400030EC16F196AF2BEEC
:1086A000198EF29EF20E0101396F0001D1EC10F02B
:1086B00019BEF28EC12FF2D793800400070E006E10
:1086C000002EFED700D0938081B01DD0FC0EF66E38
:1086D000110EF76E196AF2BE198EF29EB4EC11F00B
:1086E00019BEF28E020EC16F196AF2BE198EF29E89
:1086F000FA0E0101396F0001FEEC19F019BEF28E7D
:10870000C12FF2D765D004006B0E006E002EFED78D
:1087100000D09380C09181A0C0810400196AF2BE8C
:10872000198EF29EEF0E0101396F0001D1EC10F0AD
:1087300019BEF28EC0A101D0BF2BBE2BA7D7010E50
:10874000BE5DC16F2A0EF66E120EF76E196AF2BE8A
:10875000198EF29E090E0101396F0001EAEC13F047
:1087600019BEF28E196AF2BE198EF29EC1C038F19E
:108770001B0E0101396F000143EC11F019BEF28E9E
:10878000350EF66E120EF76E196AF2BE198EF29E53
:10879000070E0101396F0001EAEC13F019BEF28EE9
:1087A000196AF2BE198EF29EBFC038F11B0E01018C
:1087B000396F000143EC11F019BEF28E0D0E04006A
:1087C0009EA8FDD7AD6E0A0E04009EA8FDD7AD6E23
:1087D000A1EF54F0C76BC86B010EC96FDA6AD96A92
:1087E000CC6BBF0ECB6FEA6AC30EE96ECCC0E2FF62
:1087F000CBC0E1FFC9C0CAF0D890E550EE02F350FB
:10880000C723F450C823CA2FF7D7C7C0DEFFC8C09C
:10881000C7F0C86BD8B0C82BCB2BD8B4CC2BC92B86
:10882000C9510508E0E18CEF46F018EC11F0196A27
:10883000F2BE198EF29E010E0101356F250E366FC4
:10884000280E376F000185EC11F019BEF28E500E24
:10885000F66E1C0EF76E196AF2BE198EF29EB4EC1B
:1088600011F019BEF28E196AF2BE198EF29EC6EC94
:1088700011F019BEF28E7A0EF66E1C0EF76E196AA2
:10888000F2BE198EF29EB4EC11F019BEF28E7A0E81
:10889000F66E0E0EF76E196AF2BE198EF29EB4ECE9
:1088A00011F019BEF28EC20EF66E0E0EF76E196A38
:1088B000F2BE198EF29EB4EC11F019BEF28E0A0EC1
:1088C000F66E0F0EF76E196AF2BE198EF29EB4ECB8
:1088D00011F019BEF28E520EF66E0F0EF76E196A77
:1088E000F2BE198EF29EB4EC11F019BEF28E9A0E01
:1088F000F66E0F0EF76E196AF2BE198EF29EB4EC88
:1089000011F019BEF28EA40EF66E1C0EF76E196AE7
:10891000F2BE198EF29EB4EC11F019BEF28E79EC13
:1089200026F001C0BEF0196AF2BE198EF29E010E49
:108930000101356F250E366F280E376F000185EC6B
:1089400011F019BEF28E246A236A226A216AB80ED7
:10895000F66E1C0EF76E196AF2BE198EF29EB4EC1A
:1089600011F019BEF28EBE511EE0010A29E0030A81
:1089700034E0010A3FE0070A4AE0010A55E0030A31
:1089800060E0010A6BE00F0AD8B475D0010AD8B4D0
:1089900084D0030AD8B494D0010AD8B4A4D0070A6A
:1089A000D8B4B3D0BFD0C20EF66E1C0EF76E196AE3
:1089B000F2BE198EF29EB4EC11F019BEF28EC1D047
:1089C000CC0EF66E1C0EF76E196AF2BE198EF29E70
:1089D000B4EC11F019BEF28EB4D0D60EF66E1C0EA9
:1089E000F76E196AF2BE198EF29EB4EC11F019BE40
:1089F000F28EA7D0DE0EF66E1C0EF76E196AF2BE6E
:108A0000198EF29EB4EC11F019BEF28E9AD0EA0ED5
:108A1000F66E1C0EF76E196AF2BE198EF29EB4EC59
:108A200011F019BEF28E8DD0F60EF66E1C0EF76E9A
:108A3000196AF2BE198EF29EB4EC11F019BEF28ED4
:108A400080D0020EF66E1D0EF76E196AF2BE198EF8
:108A5000F29EB4EC11F019BEF28E73D00E0EF66ECB
:108A60001D0EF76E196AF2BE198EF29EB4EC11F06B
:108A700019BEF28E66D01A0EF66E1D0EF76E196ACA
:108A8000F2BE198EF29EB4EC11F019BEF28E246A79
:108A9000236A226ADC0E216E54D02A0EF66E1D0E59
:108AA000F76E196AF2BE198EF29EB4EC11F019BE7F
:108AB000F28E246A236A020E226E580E216E41D075
:108AC0003A0EF66E1D0EF76E196AF2BE198EF29E00
:108AD000B4EC11F019BEF28E246A236A020E226EE3
:108AE000580E216E2ED04E0EF66E1D0EF76E196AC0
:108AF000F2BE198EF29EB4EC11F019BEF28E246A09
:108B0000236A226ADC0E216E1CD05E0EF66E1D0EEC
:108B1000F76E196AF2BE198EF29EB4EC11F019BE0E
:108B2000F28E0FD06A0EF66E1D0EF76E196AF2BE47
:108B3000198EF29EB4EC11F019BEF28E010EBE6FCA
:108B400000D0196AF2BE198EF29EC6EC11F019BE61
:108B5000F28EAA6A150EA96EBEC0A8FFA69CA69E9C
:108B6000A684F250006EF29E0F01550EA76EAA0E5B
:108B7000A76EA682A6B2FED7A6940050F212BEC07F
:108B80001CF0215206E1225204E1235202E1245258
:108B900001E0A9D0740EF66E1D0EF76E196AF2BED2
:108BA000198EF29E0001B4EC11F019BEF28EC40EC3
:108BB000F66E1D0EF76E196AF2BE198EF29EB4ECB7
:108BC00011F019BEF28E196AF2BE198EF29E010ED4
:108BD0000101356F250E366F280E376F000185ECC9
:108BE00011F019BEF28ECCEC38F001C000F002C0DA
:108BF00001F0026A036A03C024F002C023F001C03E
:108C000022F000C021F0196AF2BE198EF29EC6EC65
:108C100011F019BEF28E215265E1225263E1235216
:108C200061E124525FE1BE51F30F5CE20D0F10EFE2
:108C300047F0246A236A010E226EB80E216E52D0CC
:108C4000246A236A010E226EB80E216E4BD0246A6C
:108C5000236A010E226EB80E216E44D0246A236A64
:108C6000010E226EB80E216E3DD0246A236A020ED8
:108C7000226E580E216E36D0246A236A070E226EA9
:108C8000D00E216E2FD0246A236A070E226ED00EDA
:108C9000216E28D0246A236A010E226EB80E216E3E
:108CA00021D0246A236A226ADC0E216E1BD0246A3A
:108CB000236A020E226E580E216E14D0246A236A93
:108CC000020E226E580E216E0DD0246A236A226A8B
:108CD000DC0E216E07D0246A236A010E226EB80EC4
:108CE000216E00D00F012150DD0807E12250260837
:108CF00004E1235202E1245219E024C0C2F023C04F
:108D0000C1F022C0C0F021C0BFF00001C66BC56B2E
:108D1000C46B0A0EC36F5ED503C024F002C023F0FB
:108D200001C022F000C021F029D00F011A9EF00EE0
:108D3000F66E1D0EF76E196AF2BE198EF29E0001D4
:108D4000B4EC11F019BEF28EFA0EF66E1D0EF76E2F
:108D5000196AF2BE198EF29EB4EC11F019BEF28EB1
:108D60004C0EF66E1E0EF76E196AF2BE198EF29E4A
:108D7000B4EC11F019BEF28ED4EC34F023C0C0F084
:108D800024C0C1F0C26BC36BAA6A160EA96EC0C024
:108D9000A8FFA69CA69EA684F250006EF29E0F012C
:108DA000550EA76EAA0EA76EA682A6B2FED7A694EF
:108DB0000050F21222C0C0F023C0C1F024C0C2F0A3
:108DC0000001C36BAA6A170EA96EC0C0A8FFA69CBB
:108DD000A69EA684F250006EF29E0F01550EA76E5D
:108DE000AA0EA76EA682A6B2FED7A6940050F212D3
:108DF000AA6A180EA96E21C0A8FFA69CA69EA684EA
:108E0000F2CF00F0F29E550EA76EAA0EA76EA682B4
:108E1000A6B2FED7A6940050F2120001B8EF54F0AB
:108E2000E824F76AF7363B0FF66E8E0EF7220A003B
:108E3000F550FA6E0800F550F96E328C408C4E8C6D
:108E40005C8C6A8C788C868C948CA28CAE8CBC8C5E
:108E5000CA8CD68CAA0EF66E1A0EF76E196AF2BE7E
:108E6000198EF29EB4EC11F019BEF28E04009EAA87
:108E7000FDD7AE50DC0EF66E1A0EF76E196AF2BE12
:108E8000198EF29EB4EC11F019BEF28EA53D01D000
:108E900009D0196AF2BE198EF29EB9EC1AF019BE09
:108EA000F28E23D0196AF2BE198EF29E16EC1AF0D9
:108EB00019BEF28E0152F6E00400196AF2BE198E54
:108EC000F29EDD0E0101396F0001D1EC10F019BEE8
:108ED000F28E196AF2BE198EF29ECC0E0101376F26
:108EE000000180EC1AF019BEF28E0400090E006E2B
:108EF000002EFED70000196AF2BE198EF29EF00E07
:108F00000101376F000180EC1AF019BEF28E0400E7
:108F1000090E006E002EFED70000196AF2BE198EEF
:108F2000F29E0101376B000180EC1AF019BEF28E3F
:108F3000BE6BBE511F0820E30400090E006E002E18
:108F4000FED70000036ABE51BF0F016E000E032260
:108F500001C0EFF003C0F0F0196AF2BE198EF29E64
:108F6000F9EC1AF019BEF28EF0C0EAFFEFC0E9FF8B
:108F700001C0EFFFBE2BDDD7196AF2BE198EF29E3B
:108F8000040E0101396F0001FEEC19F019BEF28EDA
:108F9000196AF2BE198EF29E16EC1AF019BEF28E04
:108FA0000152F6E00400020EEF6F196AF2BE198E4C
:108FB000F29ED10E0101396F0001D1EC10F019BE03
:108FC000F28EEF2FF2D7196AF2BE198EF29E330E8F
:108FD0000101376F000180EC1AF019BEF28E200EED
:108FE000BE6FBE51270820E30400090E006E002E5C
:108FF000FED70000036ABE51BF0F016E000E0322B0
:1090000001C0EFF003C0F0F0196AF2BE198EF29EB3
:10901000F9EC1AF019BEF28EF0C0EAFFEFC0E9FFDA
:1090200001C0EFFFBE2BDDD7196AF2BE198EF29E8A
:10903000060E0101396F0001FEEC19F019BEF28E27
:10904000A53D01D009D0196AF2BE198EF29EB9EC85
:109050001AF019BEF28E23D0196AF2BE198EF29E52
:1090600016EC1AF019BEF28E0152F6E00400196AED
:10907000F2BE198EF29EDD0E0101396F0001D1ECB6
:1090800010F019BEF28E196AF2BE198EF29ECC0E45
:109090000101376F000180EC1AF019BEF28E040056
:1090A000090E006E002EFED70000196AF2BE198E5E
:1090B000F29EC30E0101376F000180EC1AF019BE59
:1090C000F28E0400090E006E002EFED70000196A11
:1090D000F2BE198EF29E0101376B000180EC1AF08E
:1090E00019BEF28E280EBE6FBE512F0820E3040079
:1090F000090E006E002EFED70000036ABE51BF0F9E
:10910000016E000E032201C0EFF003C0F0F0196AF7
:10911000F2BE198EF29EF9EC1AF019BEF28EF0C072
:10912000EAFFEFC0E9FF01C0EFFFBE2BDDD7BE6B4A
:10913000BE512F0827E3BE51EF6F010EF06F036A97
:10914000BE51BF0FE96E000E0320EA6EEFCFF1F0C3
:10915000F0C0AAFFEFC0A9FFF1C0A8FFA69CA69E81
:10916000A684F250006EF29E0F01550EA76EAA0E55
:10917000A76EA682A6B2FED7A6940050F2120001F6
:10918000BE2BD6D7FE0EF66E1A0EF76E196AF2BE19
:10919000198EF29EB4EC11F019BEF28ECBEF54F0A2
:1091A000BE6BBE512F081BE3036ABE51BF0FE96EB1
:1091B000000E0320EA6EBE51F26F010EF36FF2CF84
:1091C000F4F0F29EF3C0AAFFF2C0A9FFA69CA69EEF
:1091D000A680A850F4BFF28EEF6EBE2BE2D71ABE67
:1091E00095D00C0EF66E1B0EF76E196AF2BE198E34
:1091F000F29EB4EC11F019BEF28E2EEC25F0196A35
:10920000F2BE198EF29E16EC1AF019BEF28E0152C1
:10921000F6E0196AF2BE198EF29E990E0101376FBF
:10922000000180EC1AF019BEF28E0400200E006ED0
:10923000002EFED700D0BE6BBE512F0866E3036A36
:10924000BE51BF0FE96E000E0320EA6EEFCFF0F0C3
:10925000196AF2BE198EF29EF0C037F180EC1AF056
:1092600019BEF28E0400100E006E002EFED7196A91
:10927000F2BE198EF29EF9EC1AF019BEF28E01C000
:10928000EFF0036ABE51BF0FE96E000E0320EA6ED5
:10929000EF50EF5D31E1196AF2BE198EF29E770E42
:1092A0000101376F000180EC1AF019BEF28E3EEC1E
:1092B00025F0196AF2BE198EF29EBEC03AF1370E41
:1092C00001013B6F00011BEC1BF019BEF28E196A05
:1092D000F2BE198EF29E040E0101396F0001FEEC00
:1092E00019F019BEF28E196AF2BE198EF29EF9ECCF
:1092F0001AF019BEF28E07D00400200E006E002E68
:10930000FED700D09CD7BE2B97D74ED0BE6BBE5198
:109310001F0819E3036ABE51250F016E000E0322D8
:1093200003C0F1F0036ABE51BF0FE96E000E0320C7
:10933000EA6EEFCFF2F0F1C0EAFF01C0E9FFF2C040
:10934000EFFFBE2BE4D7BE6BBE511F0816E3FC6BCC
:10935000BEC0FDF0080EFE6FFDEC27F0196AF2BEEC
:10936000198EF29E010E0101396F0001FEEC19F019
:1093700019BEF28E080EBE27E7D7FC6BFDEC28F075
:10938000FAEC29F0196AF2BE198EF29E0101326BD5
:109390000001FDEC1BF019BEF28E010EFC6FFD6B9F
:1093A000FE6F4EEC25F01B92010EFC6FFD6FFE6F01
:1093B0004EEC25F01B92040EF06F196AF2BE198E66
:1093C000F29EFA0E0101396F0001FEEC19F019BE90
:1093D000F28EF02FF2D71B92040EF06F196AF2BED4
:1093E000198EF29EFA0E0101396F0001FEEC19F0A0
:1093F00019BEF28EF02FF2D7DEEF54F0FC6BFDECCD
:1094000028F0F2CFBFF0F29EAA6A130EA96EA69CB6
:10941000A69EA680A850BFBFF28E316EF2CFBFF0DD
:10942000F29EAA6A140EA96EA69CA69EA680A850BB
:10943000BFBFF28E326E436ABE6BBE511D080BE396
:10944000036ABE51250FE96E000E0320EA6EEF504D
:109450004326BE2BF2D7FC6B0C0EFD6F020EFE6F87
:10946000FDEC27F0FC6B1E0EFD6F010EFE6FFDEC98
:1094700027F0FAEC29F0C40EF66E1B0EF76E196A8F
:10948000F2BE198EF29EB4EC11F019BEF28E080EE7
:10949000BF6F196AF2BE198EF29EFA0E0101396F82
:1094A0000001FEEC19F019BEF28EBF2FF2D71EEFAD
:1094B00055F0196AF2BE198EF29E16EC1AF019BE1A
:1094C000F28E0152F6E00400020ECC6F196AF2BE71
:1094D000198EF29ED10E0101396F0001D1EC10F00E
:1094E00019BEF28ECC2FF2D7196AF2BE198EF29EF7
:1094F000980E0101376F000180EC1AF019BEF28E50
:10950000C46BC451020820E30400070E006E002E55
:10951000FED700D0036AC451C50F016E000E0322AE
:1095200001C0CCF003C0CDF0196AF2BE198EF29ED4
:10953000F9EC1AF019BEF28ECDC0EAFFCCC0E9FFFB
:1095400001C0EFFFC42BDDD7CB6BC5C0CAF0C6C0CE
:10955000C9F0C7C0C8F0C8C000F0C9C001F0CAC097
:1095600002F0CBC003F04EEF4BF018EC11F0196A8B
:10957000F2BE198EF29E010E0101356F250E366F77
:10958000280E376F000185EC11F019BEF28E4A0EDD
:10959000F66E1F0EF76E196AF2BE198EF29EB4ECCB
:1095A00011F019BEF28E196AF2BE198EF29EC6EC47
:1095B00011F019BEF28E700EF66E1F0EF76E196A5C
:1095C000F2BE198EF29EB4EC11F019BEF28E980E16
:1095D000F66E1F0EF76E196AF2BE198EF29EB4EC8B
:1095E00011F019BEF28E196AF2BE198EF29E0101B7
:1095F000326B0001FDEC1BF019BEF28E196AF2BE4F
:10960000198EF29E010E0101356F250E366F280E60
:10961000376F000185EC11F019BEF28E41C0C5F024
:1096200042C0C4F0196AF2BE198EF29E41C038F1F0
:1096300042C037F101013A6B0A0E396F000140EC6C
:109640001BF019BEF28E02C0C3F001C0C2F0000EC2
:10965000E96E196AF2BE198EF29EC3C03BF1C2C018
:109660003AF18FEC12F019BEF28EB80EF66E1F0EA4
:10967000F76E196AF2BE198EF29E040E0101396F5F
:109680000001EAEC13F019BEF28E196AF2BE198ECF
:10969000F29EC6EC11F019BEF28E0BD703C0C7F0D4
:1096A00002C0C6F001C0C5F000C0C4F0EACFC9F0E6
:1096B000E9CFC8F0D892196AF2BE198EF29E03C0A3
:1096C00045F102C044F101C043F100C042F1010183
:1096D000496B486B476B0A0E466F0001E6EC11F0D0
:1096E00019BEF28EC9C0EAFFC8C0E9FF03C0C1F0CD
:1096F00002C0C0F001C0BFF000C0BEF0BE0EF66EEA
:109700001F0EF76E196AF2BE198EF29EB4EC11F0BC
:1097100019BEF28E196AF2BE198EF29E010E010177
:10972000356F250E366F280E376F000185EC11F06E
:1097300019BEF28E060EE96E196AF2BE198EF29EFD
:10974000C1C039F1C0C038F1BFC037F1BEC036F179
:1097500030EC12F019BEF28EDE0EF66E1F0EF76EB2
:10976000196AF2BE198EF29E050E0101396F0001D1
:10977000EAEC13F019BEF28E196AF2BE198EF29E4F
:10978000C6EC11F019BEF28EE40EF66E1F0EF76EE7
:10979000196AF2BE198EF29EB4EC11F019BEF28E67
:1097A000196AF2BE198EF29E010E0101356F250E67
:1097B000366F280E376F000185EC11F019BEF28E5E
:1097C000C251BE25C46FC351BF21C56F000EC02159
:1097D000C66F000EC121C76F060EE96E196AF2BE90
:1097E000198EF29EC7C039F1C6C038F1C5C037F135
:1097F000C4C036F130EC12F019BEF28E040EF66ED3
:10980000200EF76E196AF2BE198EF29E050E010146
:10981000396F0001EAEC13F019BEF28E196AF2BE3C
:10982000198EF29EC6EC11F019BEF28E36EF55F08D
:1098300018EC11F0196AF2BE198EF29E010E0101A8
:10984000356F250E366F280E376F000185EC11F04D
:1098500019BEF28E960EF66E1E0EF76E196AF2BEE5
:10986000198EF29EB4EC11F019BEF28E196AF2BE96
:10987000198EF29EC6EC11F019BEF28EBA0EF66E7B
:109880001E0EF76E196AF2BE198EF29EB4EC11F03C
:1098900019BEF28EDE0EF66E1E0EF76E196AF2BE5D
:1098A000198EF29EB4EC11F019BEF28E196AF2BE56
:1098B000198EF29E010E0101356F250E366F280EAE
:1098C000376F000185EC11F019BEF28EF2CFC2F0B5
:1098D000F29EAA6A040EA96EA69CA69EA680A85017
:1098E000C2BFF28EC36FF2CFC4F0F29EAA6A030E1B
:1098F000A96EA69CA69EA680A850C4BFF28EC56F76
:10990000F2CFC6F0F29EAA6A020EA96EA69CA69E8F
:10991000A680A850C6BFF28EC76FF2CFC8F0F29EE5
:10992000AA6A010EA96EA69CA69EA680A850C8BFD2
:10993000F28EC96F196AF2BE198EF29EC3C03AF157
:10994000370E01013B6F00011BEC1BF019BEF28EBC
:10995000200E04009EA8FDD7AD6E196AF2BE198EC6
:10996000F29EC5C03AF1370E01013B6F00011BECBE
:109970001BF019BEF28E200E04009EA8FDD7AD6E1E
:10998000196AF2BE198EF29EC7C03AF1370E010174
:109990003B6F00011BEC1BF019BEF28E200E040081
:1099A0009EA8FDD7AD6E196AF2BE198EF29EC9C08F
:1099B0003AF1370E01013B6F00011BEC1BF019BEA1
:1099C000F28E200E04009EA8FDD7AD6E196AF2BE7D
:1099D000198EF29EC6EC11F019BEF28E020EF66ED2
:1099E0001F0EF76E196AF2BE198EF29EB4EC11F0DA
:1099F00019BEF28E0A0EF66E1F0EF76E196AF2BECF
:109A0000198EF29EB4EC11F019BEF28E196AF2BEF4
:109A1000198EF29E010E0101356F250E366F280E4C
:109A2000376F000185EC11F019BEF28E79EC26F04B
:109A300001C0BEF0BE51DD08D8B47AD0BE3BF00EF6
:109A4000BE1779EC26F001C0BFF0200E04009EA8DE
:109A5000FDD7AD6EBF51BE139BEC26F001C0BFF029
:109A6000200E04009EA8FDD7AD6E9BEC26F001C031
:109A7000C0F0200E04009EA8FDD7AD6E9BEC26F032
:109A800001C0C1F0AA6A040EA96EBEC0A8FFA69CC0
:109A9000A69EA684F250006EF29E0F01550EA76E90
:109AA000AA0EA76EA682A6B2FED7A6940050F21206
:109AB000AA6A030EA96EBFC0A8FFA69CA69EA68494
:109AC000F2CF00F0F29E550EA76EAA0EA76EA682E8
:109AD000A6B2FED7A6940050F212AA6A020EA96E90
:109AE000C0C0A8FFA69CA69EA684F2CF00F0F29E5E
:109AF000550EA76EAA0EA76EA682A6B2FED7A69492
:109B00000050F212AA6A010EA96EC1C0A8FFA69C5D
:109B1000A69EA684F2CF00F0F29E550EA76EAA0E66
:109B2000A76EA682A6B2FED7A6940050F21200013C
:109B3000196AF2BE198EF29EC6EC11F019BEF28EB1
:109B40004FEF55F018EC11F0196AF2BE198EF29E23
:109B5000010E0101356F250E366F280E376F00019B
:109B600085EC11F019BEF28E240EF66E1B0EF76E08
:109B7000196AF2BE198EF29EB4EC11F019BEF28E83
:109B8000196AF2BE198EF29EC6EC11F019BEF28E61
:109B90004C0EF66E1B0EF76E196AF2BE198EF29E0F
:109BA000B4EC11F019BEF28E740EF66E1B0EF76E49
:109BB000196AF2BE198EF29EB4EC11F019BEF28E43
:109BC000196AF2BE198EF29E010E0101356F250E43
:109BD000366F280E376F000185EC11F019BEF28E3A
:109BE000CCEC38F002C0BFF001C0BEF0196AF2BE82
:109BF000198EF29EC6EC11F019BEF28E0D0E040005
:109C00009EA8FDD7AD6E0A0E04009EA8FDD7AD6ECE
:109C1000BF51070805E303E1BE51D90801E3C4D7EA
:109C2000D00EBE5DC16F070EBF59C26F020EC125B7
:109C3000BE6F000EC221BF6F980EF66E1B0EF76E40
:109C4000196AF2BE198EF29EB4EC11F019BEF28EB2
:109C5000196AF2BE198EF29E010E0101356F250EB2
:109C6000366F280E376F000185EC11F019BEF28EA9
:109C7000E8EC27F001C0C0F0196AF2BE198EF29E1E
:109C8000C6EC11F019BEF28E0D0E04009EA8FDD791
:109C9000AD6E0A0E04009EA8FDD7AD6EC05303E062
:109CA000C0510C0801E2C8D7AA6A130EA96EBEC043
:109CB000A8FFA69CA69EA684F250006EF29E0F01FD
:109CC000550EA76EAA0EA76EA682A6B2FED7A694C0
:109CD0000050F212AA6A140EA96EC0C0A8FFA69C7A
:109CE000A69EA684F2CF00F0F29E550EA76EAA0E95
:109CF000A76EA682A6B2FED7A6940050F21200016B
:109D000064EF55F0EACFCFF0E9CFCEF0C8AF08D07E
:109D1000CE8FCEA9CE2BC71FC81FC72BD8B4C82B38
:109D2000C839F009CA6FCA27E20FCB6F320FCD6F67
:109D3000C8510F0BCB27CB27CD27E90FCC6FCC27F2
:109D4000CC27C7390F0BCC27CD27CC37CD37CD1F2C
:109D5000CD37C7510F0BCD27CA37070EC96F0A0E73
:109D6000CC07CD27FDE3CB07CC27FDE3CA07CB27E4
:109D7000FDE3C907CA27FDE3EA6AC90EE96E070ECB
:109D8000CE15CE9DE906CE1507E1CEB9E92ACEB9AA
:109D900003D0200E006E1CD0E926CD0EE95CD8B4AD
:109DA000CE8DEF50006E08E1CEBD06D0CEB915D0F5
:109DB000CEB702D0200E0BD0CEAF06D02D0E006E47
:109DC000ED50CE9DCE9F04D0CE87CE99300E00268A
:109DD000005004009EA8FDD7AD6EEE50CEADDDD78D
:109DE000000C18EC11F0196AF2BE198EF29E010EE9
:109DF0000101356F250E366F280E376F000185EC97
:109E000011F019BEF28E0A0EF66E200EF76E196A68
:109E1000F2BE198EF29EB4EC11F019BEF28E196AE0
:109E2000F2BE198EF29EC6EC11F019BEF28E4C0EE7
:109E3000F66E200EF76E196AF2BE198EF29EB4EC21
:109E400011F019BEF28E8E0EF66E200EF76E196AA4
:109E5000F2BE198EF29EB4EC11F019BEF28E196AA0
:109E6000F2BE198EF29E010E0101356F250E366F7E
:109E7000280E376F000185EC11F019BEF28ECCEC84
:109E800038F002C0BFF001C0BEF0196AF2BE198EF0
:109E9000F29EC6EC11F019BEF28E196AF2BE198E4E
:109EA000F29E0101326B0001FDEC1BF019BEF28E37
:109EB00041C0C8F042C0C7F0196AF2BE198EF29EC6
:109EC00041C038F142C037F101013A6B0A0E396FD7
:109ED000000140EC1BF019BEF28E02C0C3F001C0BD
:109EE000C2F0C80EF66E200EF76E196AF2BE198E19
:109EF000F29E190E0101396F0001EAEC13F019BE50
:109F0000F28E100EE96E196AF2BE198EF29EC3C06F
:109F10003BF1C2C03AF18FEC12F019BEF28EE40EA2
:109F2000F66E200EF76E196AF2BE198EF29E040EBE
:109F30000101396F0001EAEC13F019BEF28E2C0E0C
:109F4000BE5DC06F010EBF59C16FEA0EF66E200EE6
:109F5000F76E196AF2BE198EF29E190E0101396F61
:109F60000001EAEC13F019BEF28E100EE96E196AC8
:109F7000F2BE198EF29EC1C03BF1C0C03AF18FEC27
:109F800012F019BEF28E060EF66E210EF76E196AE9
:109F9000F2BE198EF29E040E0101396F0001EAEC47
:109FA00013F019BEF28EC251C05D006EC351C1598B
:109FB00000C0C4F0C56F0C0EF66E210EF76E196A64
:109FC000F2BE198EF29E190E0101396F0001EAEC02
:109FD00013F019BEF28E100EE96EC5C0C8F0C4C0F1
:109FE000C7F090DE280EF66E210EF76E196AF2BEEB
:109FF000198EF29E040E0101396F0001EAEC13F094
:10A0000019BEF28EC45302E1C55360E0FC6BFDEC57
:10A0100028F0C1C0FDF0C0C0FCF0FF6B0A0EFE6F5F
:10A02000E4EC20F002C041F0C1C0FDF0C0C0FCF083
:10A03000FF6B0A0EFE6FE4EC20F001C042F0436AB1
:10A04000C66BC6511D080BE3036AC651250FE96EA6
:10A05000000E0320EA6EEF504326C62BF2D7FC6BAE
:10A060001C0EFD6F030EFE6FFDEC27F0FAEC29F0DD
:10A07000010EFC6FFD6BFE6F4EEC25F02E0EF66EA2
:10A08000210EF76E196AF2BE198EF29E3A0E010188
:10A09000396F0001EAEC13F019BEF28E100EE96E72
:10A0A000C5C0C8F0C4C0C7F02DDE6B0EF66E210E21
:10A0B000F76E196AF2BE198EF29E040E0101396F15
:10A0C0000001EAEC13F019BEF28E0CD0700EF66EA1
:10A0D000210EF76E196AF2BE198EF29EB4EC11F0E1
:10A0E00019BEF28E77EF55F0F86AD09E078EEA6AB5
:10A0F000E96AB8862A0EAF6E000EB06EA60EAC6E80
:10A10000900EAB6E1B901E6A1D6AFF0E206E1F6EB6
:10A110001B924E6A4D6AA56FC150C00B0F09C16EEC
:10A12000070EB46E456A466A476A486A496A4A6ACF
:10A130004B6A4C6A4F6A506AD190C150C00B0F09EC
:10A14000C16EC290C69A949A94889496010EC66E77
:10A15000000EC76ED190810ED56ECD6A000ECA6E0C
:10A16000000ECB6E070EB46E9250926E0400100E6D
:10A17000006E002EFED7B450A19CB56AF2CFBEF09F
:10A18000F29EAA6A150EA96EA69CA69EA680A8504D
:10A19000BEBFF28E1C6E1C50040817E21C6AAA6A2D
:10A1A000150EA96EA86AA69CA69EA684F250006E03
:10A1B000F29E0F01550EA76EAA0EA76EA682A6B23A
:10A1C000FED7A6940050F2120001F2CFBEF0F29E2C
:10A1D000AA6A240EA96EA69CA69EA680A850BEBF01
:10A1E000F28E1A6EF2CFBFF0F29EAA6A160EA96E18
:10A1F000A69CA69EA680A850BFBFF28EC06FF2CFCD
:10A20000C1F0F29EAA6A170EA96EA69CA69EA68011
:10A21000A850C1BFF28EC26FF2CFC3F0F29EAA6AFD
:10A22000180EA96EA69CA69EA680A850C3BFF28E4B
:10A23000C46F246AC0C023F0C2C022F0C4C021F0A1
:10A24000213C5CD0223C5AD0233C58D0243C56D0F0
:10A25000246A236A110E226E300E216E23C0BFF0D5
:10A2600024C0C0F0C16BC26BAA6A160EA96EBFC033
:10A27000A8FFA69CA69EA684F250006EF29E0F0137
:10A28000550EA76EAA0EA76EA682A6B2FED7A694FA
:10A290000050F21222C0BFF023C0C0F024C0C1F0B1
:10A2A0000001C26BAA6A170EA96EBFC0A8FFA69CC8
:10A2B000A69EA684F250006EF29E0F01550EA76E68
:10A2C000AA0EA76EA682A6B2FED7A6940050F212DE
:10A2D000AA6A180EA96E21C0A8FFA69CA69EA684F5
:10A2E000F2CF00F0F29E550EA76EAA0EA76EA682C0
:10A2F000A6B2FED7A6940050F212000160EC1FF047
:10A30000196AF2BE198EF29E640E0101396F0001C6
:10A31000FEEC19F019BEF28E63EC1FF0F2CFBEF026
:10A32000F29EAA6A240EA96EA69CA69EA680A8509C
:10A33000BEBFF28E1A6E65EF1FF071EF1FF0196A43
:10A34000F2BE198EF29E27EC18F019BEF28ED76A73
:10A35000D66AF294F28AC00EF212D18004009EAA4C
:10A36000FDD7AECFBBF0BB51600806E2BB517A0807
:10A3700003E3BB51DF0B01D0BB51BB6FBC51BB5DD5
:10A3800004E04E6A010E4D6E03D04D2AD8B44E2A19
:10A3900060EC1FF0BB51310A58E0030AD8B476D004
:10A3A000010AD8B495D0070AD8B4B4D0010AD8B4F9
:10A3B000D3D0030AD8B4F2D0010AD8B411D1760AA6
:10A3C000D8B430D1030AD8B451D1010AD8B46CD171
:10A3D000070AD8B48DD1010AD8B4A7D1030AD8B4DA
:10A3E000C0D1010AD8B419D20F0AD8B42AD2010AAE
:10A3F000D8B43DD2030AD8B453D2010AD8B467D234
:10A40000060AD8B47AD2030AD8B490D2010AD8B4D2
:10A41000A7D21F0AD8B4B7D2010AD8B4C7D2030A48
:10A42000D8B4D7D2010AD8B4FFD2070AD8B411D30E
:10A43000010AD8B42AD3030AD8B43ED3010AD8B447
:10A440004ED30F0AD8B460D36CD31BB201D074D3EF
:10A45000F29A310E04009EA8FDD7AD6E0D0E0400D9
:10A460009EA8FDD7AD6E0A0E04009EA8FDD7AD6E66
:10A47000BE6B72EC2AF0196AF2BE198EF29E27ECBE
:10A4800018F019BEF28EF294F28A56D31BB201D0A4
:10A4900053D3F29A320E04009EA8FDD7AD6E0D0E76
:10A4A00004009EA8FDD7AD6E0A0E04009EA8FDD73D
:10A4B000AD6E010EBE6F72EC2AF0196AF2BE198EF3
:10A4C000F29E27EC18F019BEF28EF294F28A34D381
:10A4D0001BB201D031D3F29A330E04009EA8FDD7EF
:10A4E000AD6E0D0E04009EA8FDD7AD6E0A0E0400E1
:10A4F0009EA8FDD7AD6E020EBE6F72EC2AF0196AEF
:10A50000F2BE198EF29E27EC18F019BEF28EF2946C
:10A51000F28A12D31BB201D00FD3F29A340E040088
:10A520009EA8FDD7AD6E0D0E04009EA8FDD7AD6EA2
:10A530000A0E04009EA8FDD7AD6E030EBE6F72EC2E
:10A540002AF0196AF2BE198EF29E27EC18F019BE95
:10A55000F28EF294F28AF0D21BB201D0EDD2F29ACE
:10A56000350E04009EA8FDD7AD6E0D0E04009EA80A
:10A57000FDD7AD6E0A0E04009EA8FDD7AD6E040E89
:10A58000BE6F72EC2AF0196AF2BE198EF29E27ECA9
:10A5900018F019BEF28EF294F28ACED21BB201D01C
:10A5A000CBD2F29A360E04009EA8FDD7AD6E0D0EEA
:10A5B00004009EA8FDD7AD6E0A0E04009EA8FDD72C
:10A5C000AD6E050EBE6F72EC2AF0196AF2BE198EDE
:10A5D000F29E27EC18F019BEF28EF294F28AACD2F9
:10A5E0001BB201D0A9D2F29A370E04009EA8FDD763
:10A5F000AD6E0D0E04009EA8FDD7AD6E0A0E0400D0
:10A600009EA8FDD7AD6E0F0EBE6F72EC2AF0196AD0
:10A61000F2BE198EF29E27EC18F019BEF28EF2945B
:10A62000F28A8AD21BB201D087D2F29A410E04007C
:10A630009EA8FDD7AD6E196AF2BE198EF29E010E6C
:10A640000101356F0001C2EC1BF019BEF28ED4EC93
:10A6500034F063EC1FF0196AF2BE198EF29E27ECFB
:10A6600018F019BEF28EF294F28A66D21BB001D0B5
:10A6700063D21BB201D060D2F29A420E04009EA8AF
:10A68000FDD7AD6EBE6B66EF36F063EC1FF0D4EC19
:10A6900034F0196AF2BE198EF29E27EC18F019BE3A
:10A6A000F28EF294F28A48D21BB201D045D2F29ACD
:10A6B000430E04009EA8FDD7AD6E196AF2BE198E36
:10A6C000F29E010E0101326F0001FDEC1BF019BE7C
:10A6D000F28E63EC1FF0D4EC34F0196AF2BE198EDE
:10A6E000F29E27EC18F019BEF28EF294F28A24D270
:10A6F0001BB001D021D21BB201D01ED2F29A440E5F
:10A7000004009EA8FDD7AD6E010EFC6FFD6BFE6BC5
:10A71000FDEC27F0196AF2BE198EF29E27EC18F0B4
:10A7200019BEF28EF294F28A07D21BB201D004D283
:10A73000F29A450E04009EA8FDD7AD6E010EFC6F87
:10A74000FDEC28F0D4EC34F063EC1FF0196AF2BE93
:10A75000198EF29E27EC18F019BEF28EF294F28A4E
:10A76000EBD1F29A460E04009EA8FDD7AD6EF2CF53
:10A77000BEF0F29EAA6A100EA96EA69CA69EA680A6
:10A78000A850BEBFF28EBF6FF2CFC0F0F29EAA6A91
:10A79000110EA96EA69CA69EA680A850C0BFF28EE0
:10A7A000C16FBFC0C3F0C1C0C2F0A00EF66E3E0EB6
:10A7B000F76E196AF2BE198EF29E190E0101396FF9
:10A7C0000001EAEC13F019BEF28E100EE96E196A60
:10A7D000F2BE198EF29EC3C03BF1C2C03AF18FECBB
:10A7E00012F019BEF28E0A0E04009EA8FDD7AD6EBF
:10A7F0000D0E04009EA8FDD7AD6ED4EC34F063ECD2
:10A800001FF0196AF2BE198EF29E27EC18F019BEDD
:10A81000F28EF294F28AD1808FD1F29A470E040020
:10A820009EA8FDD7AD6E1DEF3DF0196AF2BE198EE0
:10A83000F29E27EC18F019BEF28EF294F28AD180C3
:10A840007BD11BB201D078D1F29A480E04009EA8A9
:10A85000FDD7AD6EFAEC29F0196AF2BE198EF29EA0
:10A8600027EC18F019BEF28EF294F28A65D1F29AB2
:10A87000490E04009EA8FDD7AD6E010EBE6FAEEF6F
:10A880003FF0D4EC34F063EC1FF0196AF2BE198E7D
:10A89000F29E27EC18F019BEF28EF294F28A4CD197
:10A8A0001BB001D049D1F29A4A0E04009EA8FDD7F0
:10A8B000AD6EBE6BD9EF40F0196AF2BE198EF29EF2
:10A8C00027EC18F019BEF28EF294F28A35D11BB043
:10A8D00001D032D1F29A4B0E04009EA8FDD7AD6E86
:10A8E00073EC40F0196AF2BE198EF29E27EC18F054
:10A8F00019BEF28EF294F28A1FD1F29A4D0E040024
:10A900009EA8FDD7AD6E010EBE6F85EF42F0D4EC70
:10A9100034F063EC1FF0196AF2BE198EF29E27EC38
:10A9200018F019BEF28EF294F28A06D11BB001D053
:10A9300003D1F29A4E0E04009EA8FDD7AD6E43EFF0
:10A9400043F0D4EC34F063EC1FF0196AF2BE198EB8
:10A95000F29E27EC18F019BEF28EF294F28AECD037
:10A96000F29A4F0E04009EA8FDD7AD6E15EF44F08D
:10A97000196AF2BE198EF29E27EC18F019BEF28EFB
:10A98000F294F28AD9D0F29A500E04009EA8FDD714
:10A99000AD6E2AEF47F0196AF2BE198EF29E27ECCF
:10A9A00018F019BEF28EF294F28AC6D0F29A510EC5
:10A9B00004009EA8FDD7AD6ED0EF48F0196AF2BE34
:10A9C000198EF29E27EC18F019BEF28EF294F28ADC
:10A9D000B3D0F29A520E04009EA8FDD7AD6E1A7E37
:10A9E0001AC0BDF0AA6A240EA96EBDC0A8FFA69C1D
:10A9F000A69EA684F250006EF29E0F01550EA76E21
:10AA0000AA0EA76EA682A6B2FED7A6940050F21296
:10AA1000196AF2BE198EF29E000127EC18F019BED9
:10AA2000F28EF294F28A88D01BB201D085D0530EF8
:10AA300004009EA8FDD7AD6EFEEF49F0196AF2BE84
:10AA4000198EF29E27EC18F019BEF28EF294F28A5B
:10AA500073D01BB001D070D01BB201D06DD0540E9A
:10AA600004009EA8FDD7AD6EB5EF4AF0D4EC34F0EB
:10AA700063EC1FF0196AF2BE198EF29E27EC18F0F3
:10AA800019BEF28EF294F28A57D01BB001D054D086
:10AA9000550E04009EA8FDD7AD6E18EF4CF063EC88
:10AAA0001FF0196AF2BE198EF29E27EC18F019BE3B
:10AAB000F28EF294F28A40D0F29A560E04009EA8CA
:10AAC000FDD7AD6EA2EF4DF0196AF2BE198EF29E5F
:10AAD00027EC18F019BEF28EF294F28A2DD0F29A79
:10AAE000570E04009EA8FDD7AD6EF1EF4EF0D4ECEA
:10AAF00034F0196AF2BE198EF29E27EC18F019BED6
:10AB0000F28EF294F28A18D0F29A1B70196AF2BE91
:10AB1000198EF29E27EC18F019BEF28EF294F28A8A
:10AB20000BD00D0E04009EA8FDD7AD6E0A0E0400DA
:10AB30009EA8FDD7AD6E00D063EC1FF0BBC0BCF08B
:04AB40000DD403002D
:020000040030CA
:0E00000000C20E1E00858100000007A0070050
:00000001FF
